

Microchip Technology PIC LITE Macro Assembler V1.12 build 49521 
                                                                                               Tue Dec 30 21:05:02 2014

HI-TECH Software Omniscient Code Generator (Lite mode) build 49521
     1  0000                     opt subtitle "HI-TECH Software Omniscient Code Generator (Lite mode) build 49521"
     2                           opt subtitle "HI-TECH Software Omniscient Code Generator (Lite mode) build 49521"
     3                           
     4                           opt pagewidth 120
     5                           
     6                           	opt lm
     7                           
     8                           	processor	16F877A
     9                           clrc	macro
    10  0000                     	endm
    11                           opt subtitle "HI-TECH Software Omniscient Code Generator (Lite mode) build 49521"
    12                           
    13  0000                     	endm
    14                           opt subtitle "HI-TECH Software Omniscient Code Generator (Lite mode) build 49521"
    15                           
    16  0000                     	endm
    17                           opt subtitle "HI-TECH Software Omniscient Code Generator (Lite mode) build 49521"
    18                           
    19  0000                     	endm
    20                           opt subtitle "HI-TECH Software Omniscient Code Generator (Lite mode) build 49521"
    21                           
    22  0000                     	endm
    23                           opt subtitle "HI-TECH Software Omniscient Code Generator (Lite mode) build 49521"
    24                           
    25  0000                     	endm
    26                           opt subtitle "HI-TECH Software Omniscient Code Generator (Lite mode) build 49521"
    27                           
    28  0000                     	endm
    29                           opt subtitle "HI-TECH Software Omniscient Code Generator (Lite mode) build 49521"
    30                           
    31  0000                     	endm
    32  0000                     indf	equ	0
    33  0000                     indf0	equ	0
    34  0002                     pc	equ	2
    35  0002                     pcl	equ	2
    36  0003                     status	equ	3
    37  0004                     fsr	equ	4
    38  0004                     fsr0	equ	4
    39  0001                     c	equ	1
    40  0000                     z	equ	0
    41  000A                     pclath	equ	10
    42                           opt subtitle "HI-TECH Software Omniscient Code Generator (Lite mode) build 49521"
    43  0000                     INDF equ 00h ;# 
    44                           opt subtitle "HI-TECH Software Omniscient Code Generator (Lite mode) build 49521"
    45  0001                     TMR0 equ 01h ;# 
    46                           opt subtitle "HI-TECH Software Omniscient Code Generator (Lite mode) build 49521"
    47  0002                     PCL equ 02h ;# 
    48                           opt subtitle "HI-TECH Software Omniscient Code Generator (Lite mode) build 49521"
    49  0003                     STATUS equ 03h ;# 
    50                           opt subtitle "HI-TECH Software Omniscient Code Generator (Lite mode) build 49521"
    51  0004                     FSR equ 04h ;# 
    52                           opt subtitle "HI-TECH Software Omniscient Code Generator (Lite mode) build 49521"
    53  0005                     PORTA equ 05h ;# 
    54                           opt subtitle "HI-TECH Software Omniscient Code Generator (Lite mode) build 49521"
    55  0006                     PORTB equ 06h ;# 
    56                           opt subtitle "HI-TECH Software Omniscient Code Generator (Lite mode) build 49521"
    57  0007                     PORTC equ 07h ;# 
    58                           opt subtitle "HI-TECH Software Omniscient Code Generator (Lite mode) build 49521"
    59  0008                     PORTD equ 08h ;# 
    60                           opt subtitle "HI-TECH Software Omniscient Code Generator (Lite mode) build 49521"
    61  0009                     PORTE equ 09h ;# 
    62                           opt subtitle "HI-TECH Software Omniscient Code Generator (Lite mode) build 49521"
    63  000A                     PCLATH equ 0Ah ;# 
    64                           opt subtitle "HI-TECH Software Omniscient Code Generator (Lite mode) build 49521"
    65  000B                     INTCON equ 0Bh ;# 
    66                           opt subtitle "HI-TECH Software Omniscient Code Generator (Lite mode) build 49521"
    67  000C                     PIR1 equ 0Ch ;# 
    68                           opt subtitle "HI-TECH Software Omniscient Code Generator (Lite mode) build 49521"
    69  000D                     PIR2 equ 0Dh ;# 
    70                           opt subtitle "HI-TECH Software Omniscient Code Generator (Lite mode) build 49521"
    71  000E                     TMR1 equ 0Eh ;# 
    72                           opt subtitle "HI-TECH Software Omniscient Code Generator (Lite mode) build 49521"
    73  000E                     TMR1L equ 0Eh ;# 
    74                           opt subtitle "HI-TECH Software Omniscient Code Generator (Lite mode) build 49521"
    75  000F                     TMR1H equ 0Fh ;# 
    76                           opt subtitle "HI-TECH Software Omniscient Code Generator (Lite mode) build 49521"
    77  0010                     T1CON equ 010h ;# 
    78                           opt subtitle "HI-TECH Software Omniscient Code Generator (Lite mode) build 49521"
    79  0011                     TMR2 equ 011h ;# 
    80                           opt subtitle "HI-TECH Software Omniscient Code Generator (Lite mode) build 49521"
    81  0012                     T2CON equ 012h ;# 
    82                           opt subtitle "HI-TECH Software Omniscient Code Generator (Lite mode) build 49521"
    83  0013                     SSPBUF equ 013h ;# 
    84                           opt subtitle "HI-TECH Software Omniscient Code Generator (Lite mode) build 49521"
    85  0014                     SSPCON equ 014h ;# 
    86                           opt subtitle "HI-TECH Software Omniscient Code Generator (Lite mode) build 49521"
    87  0015                     CCPR1 equ 015h ;# 
    88                           opt subtitle "HI-TECH Software Omniscient Code Generator (Lite mode) build 49521"
    89  0015                     CCPR1L equ 015h ;# 
    90                           opt subtitle "HI-TECH Software Omniscient Code Generator (Lite mode) build 49521"
    91  0016                     CCPR1H equ 016h ;# 
    92                           opt subtitle "HI-TECH Software Omniscient Code Generator (Lite mode) build 49521"
    93  0017                     CCP1CON equ 017h ;# 
    94                           opt subtitle "HI-TECH Software Omniscient Code Generator (Lite mode) build 49521"
    95  0018                     RCSTA equ 018h ;# 
    96                           opt subtitle "HI-TECH Software Omniscient Code Generator (Lite mode) build 49521"
    97  0019                     TXREG equ 019h ;# 
    98                           opt subtitle "HI-TECH Software Omniscient Code Generator (Lite mode) build 49521"
    99  001A                     RCREG equ 01Ah ;# 
   100                           opt subtitle "HI-TECH Software Omniscient Code Generator (Lite mode) build 49521"
   101  001B                     CCPR2 equ 01Bh ;# 
   102                           opt subtitle "HI-TECH Software Omniscient Code Generator (Lite mode) build 49521"
   103  001B                     CCPR2L equ 01Bh ;# 
   104                           opt subtitle "HI-TECH Software Omniscient Code Generator (Lite mode) build 49521"
   105  001C                     CCPR2H equ 01Ch ;# 
   106                           opt subtitle "HI-TECH Software Omniscient Code Generator (Lite mode) build 49521"
   107  001D                     CCP2CON equ 01Dh ;# 
   108                           opt subtitle "HI-TECH Software Omniscient Code Generator (Lite mode) build 49521"
   109  001E                     ADRESH equ 01Eh ;# 
   110                           opt subtitle "HI-TECH Software Omniscient Code Generator (Lite mode) build 49521"
   111  001F                     ADCON0 equ 01Fh ;# 
   112                           opt subtitle "HI-TECH Software Omniscient Code Generator (Lite mode) build 49521"
   113  0081                     OPTION_REG equ 081h ;# 
   114                           opt subtitle "HI-TECH Software Omniscient Code Generator (Lite mode) build 49521"
   115  0085                     TRISA equ 085h ;# 
   116                           opt subtitle "HI-TECH Software Omniscient Code Generator (Lite mode) build 49521"
   117  0086                     TRISB equ 086h ;# 
   118                           opt subtitle "HI-TECH Software Omniscient Code Generator (Lite mode) build 49521"
   119  0087                     TRISC equ 087h ;# 
   120                           opt subtitle "HI-TECH Software Omniscient Code Generator (Lite mode) build 49521"
   121  0088                     TRISD equ 088h ;# 
   122                           opt subtitle "HI-TECH Software Omniscient Code Generator (Lite mode) build 49521"
   123  0089                     TRISE equ 089h ;# 
   124                           opt subtitle "HI-TECH Software Omniscient Code Generator (Lite mode) build 49521"
   125  008C                     PIE1 equ 08Ch ;# 
   126                           opt subtitle "HI-TECH Software Omniscient Code Generator (Lite mode) build 49521"
   127  008D                     PIE2 equ 08Dh ;# 
   128                           opt subtitle "HI-TECH Software Omniscient Code Generator (Lite mode) build 49521"
   129  008E                     PCON equ 08Eh ;# 
   130                           opt subtitle "HI-TECH Software Omniscient Code Generator (Lite mode) build 49521"
   131  0091                     SSPCON2 equ 091h ;# 
   132                           opt subtitle "HI-TECH Software Omniscient Code Generator (Lite mode) build 49521"
   133  0092                     PR2 equ 092h ;# 
   134                           opt subtitle "HI-TECH Software Omniscient Code Generator (Lite mode) build 49521"
   135  0093                     SSPADD equ 093h ;# 
   136                           opt subtitle "HI-TECH Software Omniscient Code Generator (Lite mode) build 49521"
   137  0094                     SSPSTAT equ 094h ;# 
   138                           opt subtitle "HI-TECH Software Omniscient Code Generator (Lite mode) build 49521"
   139  0098                     TXSTA equ 098h ;# 
   140                           opt subtitle "HI-TECH Software Omniscient Code Generator (Lite mode) build 49521"
   141  0099                     SPBRG equ 099h ;# 
   142                           opt subtitle "HI-TECH Software Omniscient Code Generator (Lite mode) build 49521"
   143  009C                     CMCON equ 09Ch ;# 
   144                           opt subtitle "HI-TECH Software Omniscient Code Generator (Lite mode) build 49521"
   145  009D                     CVRCON equ 09Dh ;# 
   146                           opt subtitle "HI-TECH Software Omniscient Code Generator (Lite mode) build 49521"
   147  009E                     ADRESL equ 09Eh ;# 
   148                           opt subtitle "HI-TECH Software Omniscient Code Generator (Lite mode) build 49521"
   149  009F                     ADCON1 equ 09Fh ;# 
   150                           opt subtitle "HI-TECH Software Omniscient Code Generator (Lite mode) build 49521"
   151  010C                     EEDATA equ 010Ch ;# 
   152                           opt subtitle "HI-TECH Software Omniscient Code Generator (Lite mode) build 49521"
   153  010D                     EEADR equ 010Dh ;# 
   154                           opt subtitle "HI-TECH Software Omniscient Code Generator (Lite mode) build 49521"
   155  010E                     EEDATH equ 010Eh ;# 
   156                           opt subtitle "HI-TECH Software Omniscient Code Generator (Lite mode) build 49521"
   157  010F                     EEADRH equ 010Fh ;# 
   158                           opt subtitle "HI-TECH Software Omniscient Code Generator (Lite mode) build 49521"
   159  018C                     EECON1 equ 018Ch ;# 
   160                           opt subtitle "HI-TECH Software Omniscient Code Generator (Lite mode) build 49521"
   161  018D                     EECON2 equ 018Dh ;# 
   162                           opt subtitle "HI-TECH Software Omniscient Code Generator (Lite mode) build 49521"
   163  0000                     INDF equ 00h ;# 
   164                           opt subtitle "HI-TECH Software Omniscient Code Generator (Lite mode) build 49521"
   165  0001                     TMR0 equ 01h ;# 
   166                           opt subtitle "HI-TECH Software Omniscient Code Generator (Lite mode) build 49521"
   167  0002                     PCL equ 02h ;# 
   168                           opt subtitle "HI-TECH Software Omniscient Code Generator (Lite mode) build 49521"
   169  0003                     STATUS equ 03h ;# 
   170                           opt subtitle "HI-TECH Software Omniscient Code Generator (Lite mode) build 49521"
   171  0004                     FSR equ 04h ;# 
   172                           opt subtitle "HI-TECH Software Omniscient Code Generator (Lite mode) build 49521"
   173  0005                     PORTA equ 05h ;# 
   174                           opt subtitle "HI-TECH Software Omniscient Code Generator (Lite mode) build 49521"
   175  0006                     PORTB equ 06h ;# 
   176                           opt subtitle "HI-TECH Software Omniscient Code Generator (Lite mode) build 49521"
   177  0007                     PORTC equ 07h ;# 
   178                           opt subtitle "HI-TECH Software Omniscient Code Generator (Lite mode) build 49521"
   179  0008                     PORTD equ 08h ;# 
   180                           opt subtitle "HI-TECH Software Omniscient Code Generator (Lite mode) build 49521"
   181  0009                     PORTE equ 09h ;# 
   182                           opt subtitle "HI-TECH Software Omniscient Code Generator (Lite mode) build 49521"
   183  000A                     PCLATH equ 0Ah ;# 
   184                           opt subtitle "HI-TECH Software Omniscient Code Generator (Lite mode) build 49521"
   185  000B                     INTCON equ 0Bh ;# 
   186                           opt subtitle "HI-TECH Software Omniscient Code Generator (Lite mode) build 49521"
   187  000C                     PIR1 equ 0Ch ;# 
   188                           opt subtitle "HI-TECH Software Omniscient Code Generator (Lite mode) build 49521"
   189  000D                     PIR2 equ 0Dh ;# 
   190                           opt subtitle "HI-TECH Software Omniscient Code Generator (Lite mode) build 49521"
   191  000E                     TMR1 equ 0Eh ;# 
   192                           opt subtitle "HI-TECH Software Omniscient Code Generator (Lite mode) build 49521"
   193  000E                     TMR1L equ 0Eh ;# 
   194                           opt subtitle "HI-TECH Software Omniscient Code Generator (Lite mode) build 49521"
   195  000F                     TMR1H equ 0Fh ;# 
   196                           opt subtitle "HI-TECH Software Omniscient Code Generator (Lite mode) build 49521"
   197  0010                     T1CON equ 010h ;# 
   198                           opt subtitle "HI-TECH Software Omniscient Code Generator (Lite mode) build 49521"
   199  0011                     TMR2 equ 011h ;# 
   200                           opt subtitle "HI-TECH Software Omniscient Code Generator (Lite mode) build 49521"
   201  0012                     T2CON equ 012h ;# 
   202                           opt subtitle "HI-TECH Software Omniscient Code Generator (Lite mode) build 49521"
   203  0013                     SSPBUF equ 013h ;# 
   204                           opt subtitle "HI-TECH Software Omniscient Code Generator (Lite mode) build 49521"
   205  0014                     SSPCON equ 014h ;# 
   206                           opt subtitle "HI-TECH Software Omniscient Code Generator (Lite mode) build 49521"
   207  0015                     CCPR1 equ 015h ;# 
   208                           opt subtitle "HI-TECH Software Omniscient Code Generator (Lite mode) build 49521"
   209  0015                     CCPR1L equ 015h ;# 
   210                           opt subtitle "HI-TECH Software Omniscient Code Generator (Lite mode) build 49521"
   211  0016                     CCPR1H equ 016h ;# 
   212                           opt subtitle "HI-TECH Software Omniscient Code Generator (Lite mode) build 49521"
   213  0017                     CCP1CON equ 017h ;# 
   214                           opt subtitle "HI-TECH Software Omniscient Code Generator (Lite mode) build 49521"
   215  0018                     RCSTA equ 018h ;# 
   216                           opt subtitle "HI-TECH Software Omniscient Code Generator (Lite mode) build 49521"
   217  0019                     TXREG equ 019h ;# 
   218                           opt subtitle "HI-TECH Software Omniscient Code Generator (Lite mode) build 49521"
   219  001A                     RCREG equ 01Ah ;# 
   220                           opt subtitle "HI-TECH Software Omniscient Code Generator (Lite mode) build 49521"
   221  001B                     CCPR2 equ 01Bh ;# 
   222                           opt subtitle "HI-TECH Software Omniscient Code Generator (Lite mode) build 49521"
   223  001B                     CCPR2L equ 01Bh ;# 
   224                           opt subtitle "HI-TECH Software Omniscient Code Generator (Lite mode) build 49521"
   225  001C                     CCPR2H equ 01Ch ;# 
   226                           opt subtitle "HI-TECH Software Omniscient Code Generator (Lite mode) build 49521"
   227  001D                     CCP2CON equ 01Dh ;# 
   228                           opt subtitle "HI-TECH Software Omniscient Code Generator (Lite mode) build 49521"
   229  001E                     ADRESH equ 01Eh ;# 
   230                           opt subtitle "HI-TECH Software Omniscient Code Generator (Lite mode) build 49521"
   231  001F                     ADCON0 equ 01Fh ;# 
   232                           opt subtitle "HI-TECH Software Omniscient Code Generator (Lite mode) build 49521"
   233  0081                     OPTION_REG equ 081h ;# 
   234                           opt subtitle "HI-TECH Software Omniscient Code Generator (Lite mode) build 49521"
   235  0085                     TRISA equ 085h ;# 
   236                           opt subtitle "HI-TECH Software Omniscient Code Generator (Lite mode) build 49521"
   237  0086                     TRISB equ 086h ;# 
   238                           opt subtitle "HI-TECH Software Omniscient Code Generator (Lite mode) build 49521"
   239  0087                     TRISC equ 087h ;# 
   240                           opt subtitle "HI-TECH Software Omniscient Code Generator (Lite mode) build 49521"
   241  0088                     TRISD equ 088h ;# 
   242                           opt subtitle "HI-TECH Software Omniscient Code Generator (Lite mode) build 49521"
   243  0089                     TRISE equ 089h ;# 
   244                           opt subtitle "HI-TECH Software Omniscient Code Generator (Lite mode) build 49521"
   245  008C                     PIE1 equ 08Ch ;# 
   246                           opt subtitle "HI-TECH Software Omniscient Code Generator (Lite mode) build 49521"
   247  008D                     PIE2 equ 08Dh ;# 
   248                           opt subtitle "HI-TECH Software Omniscient Code Generator (Lite mode) build 49521"
   249  008E                     PCON equ 08Eh ;# 
   250                           opt subtitle "HI-TECH Software Omniscient Code Generator (Lite mode) build 49521"
   251  0091                     SSPCON2 equ 091h ;# 
   252                           opt subtitle "HI-TECH Software Omniscient Code Generator (Lite mode) build 49521"
   253  0092                     PR2 equ 092h ;# 
   254                           opt subtitle "HI-TECH Software Omniscient Code Generator (Lite mode) build 49521"
   255  0093                     SSPADD equ 093h ;# 
   256                           opt subtitle "HI-TECH Software Omniscient Code Generator (Lite mode) build 49521"
   257  0094                     SSPSTAT equ 094h ;# 
   258                           opt subtitle "HI-TECH Software Omniscient Code Generator (Lite mode) build 49521"
   259  0098                     TXSTA equ 098h ;# 
   260                           opt subtitle "HI-TECH Software Omniscient Code Generator (Lite mode) build 49521"
   261  0099                     SPBRG equ 099h ;# 
   262                           opt subtitle "HI-TECH Software Omniscient Code Generator (Lite mode) build 49521"
   263  009C                     CMCON equ 09Ch ;# 
   264                           opt subtitle "HI-TECH Software Omniscient Code Generator (Lite mode) build 49521"
   265  009D                     CVRCON equ 09Dh ;# 
   266                           opt subtitle "HI-TECH Software Omniscient Code Generator (Lite mode) build 49521"
   267  009E                     ADRESL equ 09Eh ;# 
   268                           opt subtitle "HI-TECH Software Omniscient Code Generator (Lite mode) build 49521"
   269  009F                     ADCON1 equ 09Fh ;# 
   270                           opt subtitle "HI-TECH Software Omniscient Code Generator (Lite mode) build 49521"
   271  010C                     EEDATA equ 010Ch ;# 
   272                           opt subtitle "HI-TECH Software Omniscient Code Generator (Lite mode) build 49521"
   273  010D                     EEADR equ 010Dh ;# 
   274                           opt subtitle "HI-TECH Software Omniscient Code Generator (Lite mode) build 49521"
   275  010E                     EEDATH equ 010Eh ;# 
   276                           opt subtitle "HI-TECH Software Omniscient Code Generator (Lite mode) build 49521"
   277  010F                     EEADRH equ 010Fh ;# 
   278                           opt subtitle "HI-TECH Software Omniscient Code Generator (Lite mode) build 49521"
   279  018C                     EECON1 equ 018Ch ;# 
   280                           opt subtitle "HI-TECH Software Omniscient Code Generator (Lite mode) build 49521"
   281  018D                     EECON2 equ 018Dh ;# 
   282                           opt subtitle "HI-TECH Software Omniscient Code Generator (Lite mode) build 49521"
   283                           
   284                           opt pagewidth 120
   285                           
   286                           	opt lm
   287                           
   288                           	processor	16F877A
   289                           clrc	macro
   290                           	bcf	3,0
   291                           	endm
   292                           clrz	macro
   293                           	bcf	3,2
   294                           	endm
   295                           setc	macro
   296                           	bsf	3,0
   297                           	endm
   298                           setz	macro
   299                           	bsf	3,2
   300                           	endm
   301                           skipc	macro
   302                           	btfss	3,0
   303                           	endm
   304                           skipz	macro
   305  05BA                     __pidataBANK0:
   306                           opt subtitle "HI-TECH Software Omniscient Code Generator (Lite mode) build 49521"
   307                           
   308                           opt pagewidth 120
   309                           
   310  05BA  3454               	retlw	054h
   311  05BB  3468               	retlw	068h
   312  05BC  3469               	retlw	069h
   313  05BD  3473               	retlw	073h
   314  05BE  3420               	retlw	020h
   315  05BF  3469               	retlw	069h
   316  05C0  3473               	retlw	073h
   317  05C1  3420               	retlw	020h
   318  05C2  3461               	retlw	061h
   319  05C3  3420               	retlw	020h
   320  05C4  3474               	retlw	074h
   321  05C5  3465               	retlw	065h
   322  05C6  3473               	retlw	073h
   323  05C7  3474               	retlw	074h
   324  05C8  3400               	retlw	0
   325                           opt subtitle "HI-TECH Software Omniscient Code Generator (Lite mode) build 49521"
   326                           
   327                           opt pagewidth 120
   328  0006                     _PORTBbits	set	0x6
   329                           opt subtitle "HI-TECH Software Omniscient Code Generator (Lite mode) build 49521"
   330  0008                     _PORTD	set	0x8
   331                           opt subtitle "HI-TECH Software Omniscient Code Generator (Lite mode) build 49521"
   332  0086                     _TRISBbits	set	0x86
   333                           opt subtitle "HI-TECH Software Omniscient Code Generator (Lite mode) build 49521"
   334  0088                     _TRISD	set	0x88
   335                           opt subtitle "HI-TECH Software Omniscient Code Generator (Lite mode) build 49521"
   336                           
   337  0000                     __CFG_BOREN$OFF equ 0x0
   338                           opt subtitle "HI-TECH Software Omniscient Code Generator (Lite mode) build 49521"
   339  0000                     __CFG_CPD$OFF equ 0x0
   340                           opt subtitle "HI-TECH Software Omniscient Code Generator (Lite mode) build 49521"
   341  0000                     __CFG_WRT$OFF equ 0x0
   342                           opt subtitle "HI-TECH Software Omniscient Code Generator (Lite mode) build 49521"
   343  0000                     __CFG_FOSC$XT equ 0x0
   344                           opt subtitle "HI-TECH Software Omniscient Code Generator (Lite mode) build 49521"
   345  0000                     __CFG_WDTE$OFF equ 0x0
   346                           opt subtitle "HI-TECH Software Omniscient Code Generator (Lite mode) build 49521"
   347  0000                     __CFG_CP$OFF equ 0x0
   348                           opt subtitle "HI-TECH Software Omniscient Code Generator (Lite mode) build 49521"
   349  0000                     __CFG_LVP$ON equ 0x0
   350                           opt subtitle "HI-TECH Software Omniscient Code Generator (Lite mode) build 49521"
   351  0000                     __CFG_PWRTE$OFF equ 0x0
   352                           opt subtitle "HI-TECH Software Omniscient Code Generator (Lite mode) build 49521"
   353                           
   354                           opt pagewidth 120
   355                           
   356  061F                     start_initialization:
   357                           opt subtitle "HI-TECH Software Omniscient Code Generator (Lite mode) build 49521"
   358                           
   359  061F                     __initialization:
   360                           opt subtitle "HI-TECH Software Omniscient Code Generator (Lite mode) build 49521"
   361                           
   362  0020                     __pbssBANK0:
   363  0020                     _lcd_buffer_1:
   364  0020                            ds      16
   365                           opt subtitle "HI-TECH Software Omniscient Code Generator (Lite mode) build 49521"
   366  0030                     _lcd_buffer_2:
   367  0030                            ds      16
   368                           opt subtitle "HI-TECH Software Omniscient Code Generator (Lite mode) build 49521"
   369                           
   370                           opt pagewidth 120
   371  0056                     __pdataBANK0:
   372                           opt subtitle "HI-TECH Software Omniscient Code Generator (Lite mode) build 49521"
   373  0056                     main@F1287:
   374  0056                            ds      15
   375                           opt subtitle "HI-TECH Software Omniscient Code Generator (Lite mode) build 49521"
   376                           
   377                           opt pagewidth 120
   378                           
   379                           	opt lm
   380  05B2                     clear_ram:
   381  05B2  0064               	clrwdt			;clear the watchdog before getting into this loop
   382  05B3                     clrloop:
   383  05B3  0180               	clrf	indf		;clear RAM location pointed to by FSR
   384  05B4  0A84               	incf	fsr,f		;increment pointer
   385  05B5  0604               	xorwf	fsr,w		;XOR with final address
   386  05B6  1903               	btfsc	status,2	;have we reached the end yet?
   387  05B7  3400               	retlw	0		;all done for this memory range, return
   388  05B8  0604               	xorwf	fsr,w		;XOR again to restore value
   389  05B9  2DB3               	goto	clrloop		;do the next byte
   390                           opt subtitle "HI-TECH Software Omniscient Code Generator (Lite mode) build 49521"
   391                           
   392                           opt pagewidth 120
   393  061F  1383               	bcf	status, 7	;select IRP bank0
   394  0620  3020               	movlw	low(__pbssBANK0)
   395  0621  0084               	movwf	fsr
   396  0622  3040               	movlw	low((__pbssBANK0)+020h)
   397  0623  120A  118A  25B2   	fcall	clear_ram
              120A  118A         
   398                           opt subtitle "HI-TECH Software Omniscient Code Generator (Lite mode) build 49521"
   399                           
   400                           opt pagewidth 120
   401                           
   402  05C9                     init_fetch:
   403  05C9  087E               	movf btemp,w
   404  05CA  008A               	movwf pclath
   405  05CB  087F               	movf btemp+1,w
   406  05CC  0082               	movwf pc
   407                           opt subtitle "HI-TECH Software Omniscient Code Generator (Lite mode) build 49521"
   408                           
   409                           opt pagewidth 120
   410                           
   411                           	opt lm
   412                           
   413  05CD                     init_ram:
   414  05CD  120A  118A  25C9   	fcall init_fetch
              120A  118A         
   415  05D2  0080               	movwf indf,f
   416  05D3  0A84               	incf fsr,f
   417  05D4  0804               	movf fsr,w
   418  05D5  067D               	xorwf btemp-1,w
   419  05D6  1903               	btfsc status,2
   420  05D7  3400               	retlw 0
   421  05D8  0AFF               	incf btemp+1,f
   422  05D9  1903               	btfsc status,2
   423  05DA  0AFE               	incf btemp,f
   424  05DB  2DCD               	goto init_ram
   425                           opt subtitle "HI-TECH Software Omniscient Code Generator (Lite mode) build 49521"
   426                           
   427                           opt pagewidth 120
   428  0628  3065               	movlw low(__pdataBANK0+15)
   429  0629  00FD               	movwf btemp-1,f
   430  062A  3005               	movlw high(__pidataBANK0)
   431  062B  00FE               	movwf btemp,f
   432  062C  30BA               	movlw low(__pidataBANK0)
   433  062D  00FF               	movwf btemp+1,f
   434  062E  3056               	movlw low(__pdataBANK0)
   435  062F  0084               	movwf fsr,f
   436  0630  120A  118A  25CD   	fcall init_ram
              120A  118A         
   437                           opt subtitle "HI-TECH Software Omniscient Code Generator (Lite mode) build 49521"
   438                           
   439                           opt pagewidth 120
   440                           
   441                           	opt lm
   442  0635                     end_of_initialization:
   443  0635                     __end_of__initialization:clrf status
      + 0635  0183               	clrf	3
   444  0636  120A  118A  2E64   ljmp _main	;jump to C main() function
   445                           opt subtitle "HI-TECH Software Omniscient Code Generator (Lite mode) build 49521"
   446                           
   447  0070                     __pcstackCOMMON:
   448  0070                     ?_lcd_cmd:	; 0 bytes @ 0x0
   449  0070                     ??_lcd_cmd:	; 0 bytes @ 0x0
   450  0070                     ?_lcd_rw:	; 0 bytes @ 0x0
   451  0070                     ??_lcd_rw:	; 0 bytes @ 0x0
   452  0070                     ?_lcd_write:	; 0 bytes @ 0x0
   453  0070                     ??_lcd_write:	; 0 bytes @ 0x0
   454  0070                     ?_lcd_en:	; 0 bytes @ 0x0
   455  0070                     ?_lcd_data:	; 0 bytes @ 0x0
   456  0070                     ??_lcd_data:	; 0 bytes @ 0x0
   457                           opt subtitle "HI-TECH Software Omniscient Code Generator (Lite mode) build 49521"
   458  0070                     ?_delay_us:	; 0 bytes @ 0x0
   459  0070                     ?_api_lcd_initialize:	; 0 bytes @ 0x0
   460  0070                     ?_api_lcd_backlight:	; 0 bytes @ 0x0
   461  0070                     ??_api_lcd_backlight:	; 0 bytes @ 0x0
   462  0070                     ?_lcd_set_line:	; 0 bytes @ 0x0
   463  0070                     ?_lcd_printf:	; 0 bytes @ 0x0
   464  0070                     ?_main:	; 2 bytes @ 0x0
   465                           opt subtitle "HI-TECH Software Omniscient Code Generator (Lite mode) build 49521"
   466  0070                     api_lcd_backlight@state:	; 1 bytes @ 0x0
   467                           opt subtitle "HI-TECH Software Omniscient Code Generator (Lite mode) build 49521"
   468  0070                     lcd_rw@sel:	; 1 bytes @ 0x0
   469                           opt subtitle "HI-TECH Software Omniscient Code Generator (Lite mode) build 49521"
   470  0070                     lcd_write@databuffer:	; 1 bytes @ 0x0
   471                           opt subtitle "HI-TECH Software Omniscient Code Generator (Lite mode) build 49521"
   472  0070                     delay_us@n:	; 2 bytes @ 0x0
   473  0070                     	ds	2
   474  0072                     ??_delay_us:	; 0 bytes @ 0x2
   475                           opt subtitle "HI-TECH Software Omniscient Code Generator (Lite mode) build 49521"
   476  0072                     delay_us@i:	; 2 bytes @ 0x2
   477  0072                     	ds	2
   478  0074                     ??_lcd_en:	; 0 bytes @ 0x4
   479  0074                     ??_api_lcd_initialize:	; 0 bytes @ 0x4
   480  0074                     ??_lcd_set_line:	; 0 bytes @ 0x4
   481                           opt subtitle "HI-TECH Software Omniscient Code Generator (Lite mode) build 49521"
   482  0074                     lcd_set_line@line:	; 1 bytes @ 0x4
   483  0074                     	ds	1
   484  0075                     ??_lcd_printf:	; 0 bytes @ 0x5
   485  0075                     	ds	1
   486                           opt subtitle "HI-TECH Software Omniscient Code Generator (Lite mode) build 49521"
   487  0076                     lcd_printf@i:	; 1 bytes @ 0x6
   488  0076                     	ds	1
   489                           opt subtitle "HI-TECH Software Omniscient Code Generator (Lite mode) build 49521"
   490  0077                     ?_api_lcd_printf:	; 0 bytes @ 0x7
   491                           opt subtitle "HI-TECH Software Omniscient Code Generator (Lite mode) build 49521"
   492  0077                     api_lcd_printf@cursor:	; 1 bytes @ 0x7
   493  0077                     	ds	1
   494                           opt subtitle "HI-TECH Software Omniscient Code Generator (Lite mode) build 49521"
   495  0078                     api_lcd_printf@databuffer:	; 1 bytes @ 0x8
   496  0078                     	ds	1
   497                           opt subtitle "HI-TECH Software Omniscient Code Generator (Lite mode) build 49521"
   498  0079                     api_lcd_printf@data_length:	; 1 bytes @ 0x9
   499  0079                     	ds	1
   500  007A                     ??_api_lcd_printf:	; 0 bytes @ 0xA
   501  007A                     	ds	3
   502                           opt subtitle "HI-TECH Software Omniscient Code Generator (Lite mode) build 49521"
   503                           
   504  0040                     __pcstackBANK0:
   505                           opt subtitle "HI-TECH Software Omniscient Code Generator (Lite mode) build 49521"
   506  0040                     api_lcd_printf@line:	; 1 bytes @ 0x0
   507  0040                     	ds	1
   508                           opt subtitle "HI-TECH Software Omniscient Code Generator (Lite mode) build 49521"
   509  0041                     api_lcd_printf@i:	; 1 bytes @ 0x1
   510  0041                     	ds	1
   511                           opt subtitle "HI-TECH Software Omniscient Code Generator (Lite mode) build 49521"
   512  0042                     api_lcd_printf@j:	; 1 bytes @ 0x2
   513  0042                     	ds	1
   514  0043                     ??_main:	; 0 bytes @ 0x3
   515  0043                     	ds	4
   516                           opt subtitle "HI-TECH Software Omniscient Code Generator (Lite mode) build 49521"
   517  0047                     main@test:	; 15 bytes @ 0x7
   518  0047                     	ds	15
   519                           opt subtitle "HI-TECH Software Omniscient Code Generator (Lite mode) build 49521"
   520                           
   521                           opt pagewidth 120
   522                           
   523                           	opt lm
   524                           
   525                           	processor	16F877A
   526                           clrc	macro
   527                           	bcf	3,0
   528                           	endm
   529                           clrz	macro
   530                           	bcf	3,2
   531                           	endm
   532                           setc	macro
   533                           	bsf	3,0
   534                           	endm
   535                           setz	macro
   536                           	bsf	3,2
   537                           	endm
   538                           skipc	macro
   539                           	btfss	3,0
   540                           	endm
   541                           skipz	macro
   542                           	btfss	3,2
   543                           	endm
   544                           skipnc	macro
   545                           	btfsc	3,0
   546                           	endm
   547                           skipnz	macro
   548                           	btfsc	3,2
   549                           	endm
   550                           indf	equ	0
   551                           indf0	equ	0
   552                           pc	equ	2
   553                           pcl	equ	2
   554                           status	equ	3
   555                           fsr	equ	4
   556                           fsr0	equ	4
   557                           c	equ	1
   558                           z	equ	0
   559                           pclath	equ	10
   560                           # 46 "C:\Program Files (x86)\Microchip\xc8\v1.12\include\pic16f877a.h"
   561                           INDF equ 00h ;# 
   562                           # 52 "C:\Program Files (x86)\Microchip\xc8\v1.12\include\pic16f877a.h"
   563                           TMR0 equ 01h ;# 
   564                           # 58 "C:\Program Files (x86)\Microchip\xc8\v1.12\include\pic16f877a.h"
   565                           PCL equ 02h ;# 
   566                           # 64 "C:\Program Files (x86)\Microchip\xc8\v1.12\include\pic16f877a.h"
   567                           STATUS equ 03h ;# 
   568                           # 151 "C:\Program Files (x86)\Microchip\xc8\v1.12\include\pic16f877a.h"
   569                           FSR equ 04h ;# 
   570                           # 157 "C:\Program Files (x86)\Microchip\xc8\v1.12\include\pic16f877a.h"
   571                           PORTA equ 05h ;# 
   572                           # 206 "C:\Program Files (x86)\Microchip\xc8\v1.12\include\pic16f877a.h"
   573                           PORTB equ 06h ;# 
   574                           # 267 "C:\Program Files (x86)\Microchip\xc8\v1.12\include\pic16f877a.h"
   575                           PORTC equ 07h ;# 
   576                           # 328 "C:\Program Files (x86)\Microchip\xc8\v1.12\include\pic16f877a.h"
   577                           PORTD equ 08h ;# 
   578                           # 389 "C:\Program Files (x86)\Microchip\xc8\v1.12\include\pic16f877a.h"
   579                           PORTE equ 09h ;# 
   580                           # 420 "C:\Program Files (x86)\Microchip\xc8\v1.12\include\pic16f877a.h"
   581                           PCLATH equ 0Ah ;# 
   582                           # 439 "C:\Program Files (x86)\Microchip\xc8\v1.12\include\pic16f877a.h"
   583                           INTCON equ 0Bh ;# 
   584                           # 516 "C:\Program Files (x86)\Microchip\xc8\v1.12\include\pic16f877a.h"
   585                           PIR1 equ 0Ch ;# 
   586                           # 577 "C:\Program Files (x86)\Microchip\xc8\v1.12\include\pic16f877a.h"
   587                           PIR2 equ 0Dh ;# 
   588                           # 616 "C:\Program Files (x86)\Microchip\xc8\v1.12\include\pic16f877a.h"
   589                           TMR1 equ 0Eh ;# 
   590                           # 622 "C:\Program Files (x86)\Microchip\xc8\v1.12\include\pic16f877a.h"
   591                           TMR1L equ 0Eh ;# 
   592                           # 628 "C:\Program Files (x86)\Microchip\xc8\v1.12\include\pic16f877a.h"
   593                           TMR1H equ 0Fh ;# 
   594                           # 634 "C:\Program Files (x86)\Microchip\xc8\v1.12\include\pic16f877a.h"
   595                           T1CON equ 010h ;# 
   596                           # 708 "C:\Program Files (x86)\Microchip\xc8\v1.12\include\pic16f877a.h"
   597                           TMR2 equ 011h ;# 
   598                           # 714 "C:\Program Files (x86)\Microchip\xc8\v1.12\include\pic16f877a.h"
   599                           T2CON equ 012h ;# 
   600                           # 784 "C:\Program Files (x86)\Microchip\xc8\v1.12\include\pic16f877a.h"
   601                           SSPBUF equ 013h ;# 
   602                           # 790 "C:\Program Files (x86)\Microchip\xc8\v1.12\include\pic16f877a.h"
   603                           SSPCON equ 014h ;# 
   604                           # 859 "C:\Program Files (x86)\Microchip\xc8\v1.12\include\pic16f877a.h"
   605                           CCPR1 equ 015h ;# 
   606                           # 865 "C:\Program Files (x86)\Microchip\xc8\v1.12\include\pic16f877a.h"
   607                           CCPR1L equ 015h ;# 
   608                           # 871 "C:\Program Files (x86)\Microchip\xc8\v1.12\include\pic16f877a.h"
   609                           CCPR1H equ 016h ;# 
   610                           # 877 "C:\Program Files (x86)\Microchip\xc8\v1.12\include\pic16f877a.h"
   611                           CCP1CON equ 017h ;# 
   612                           # 934 "C:\Program Files (x86)\Microchip\xc8\v1.12\include\pic16f877a.h"
   613                           RCSTA equ 018h ;# 
   614                           # 1028 "C:\Program Files (x86)\Microchip\xc8\v1.12\include\pic16f877a.h"
   615                           TXREG equ 019h ;# 
   616                           # 1034 "C:\Program Files (x86)\Microchip\xc8\v1.12\include\pic16f877a.h"
   617                           RCREG equ 01Ah ;# 
   618                           # 1040 "C:\Program Files (x86)\Microchip\xc8\v1.12\include\pic16f877a.h"
   619                           CCPR2 equ 01Bh ;# 
   620                           # 1046 "C:\Program Files (x86)\Microchip\xc8\v1.12\include\pic16f877a.h"
   621                           CCPR2L equ 01Bh ;# 
   622                           # 1052 "C:\Program Files (x86)\Microchip\xc8\v1.12\include\pic16f877a.h"
   623                           CCPR2H equ 01Ch ;# 
   624                           # 1058 "C:\Program Files (x86)\Microchip\xc8\v1.12\include\pic16f877a.h"
   625                           CCP2CON equ 01Dh ;# 
   626                           # 1115 "C:\Program Files (x86)\Microchip\xc8\v1.12\include\pic16f877a.h"
   627                           ADRESH equ 01Eh ;# 
   628                           # 1121 "C:\Program Files (x86)\Microchip\xc8\v1.12\include\pic16f877a.h"
   629                           ADCON0 equ 01Fh ;# 
   630                           # 1216 "C:\Program Files (x86)\Microchip\xc8\v1.12\include\pic16f877a.h"
   631                           OPTION_REG equ 081h ;# 
   632                           # 1285 "C:\Program Files (x86)\Microchip\xc8\v1.12\include\pic16f877a.h"
   633                           TRISA equ 085h ;# 
   634                           # 1334 "C:\Program Files (x86)\Microchip\xc8\v1.12\include\pic16f877a.h"
   635                           TRISB equ 086h ;# 
   636                           # 1395 "C:\Program Files (x86)\Microchip\xc8\v1.12\include\pic16f877a.h"
   637                           TRISC equ 087h ;# 
   638                           # 1456 "C:\Program Files (x86)\Microchip\xc8\v1.12\include\pic16f877a.h"
   639                           TRISD equ 088h ;# 
   640                           # 1517 "C:\Program Files (x86)\Microchip\xc8\v1.12\include\pic16f877a.h"
   641                           TRISE equ 089h ;# 
   642                           # 1573 "C:\Program Files (x86)\Microchip\xc8\v1.12\include\pic16f877a.h"
   643                           PIE1 equ 08Ch ;# 
   644                           # 1634 "C:\Program Files (x86)\Microchip\xc8\v1.12\include\pic16f877a.h"
   645                           PIE2 equ 08Dh ;# 
   646                           # 1673 "C:\Program Files (x86)\Microchip\xc8\v1.12\include\pic16f877a.h"
   647                           PCON equ 08Eh ;# 
   648                           # 1706 "C:\Program Files (x86)\Microchip\xc8\v1.12\include\pic16f877a.h"
   649                           SSPCON2 equ 091h ;# 
   650                           # 1767 "C:\Program Files (x86)\Microchip\xc8\v1.12\include\pic16f877a.h"
   651                           PR2 equ 092h ;# 
   652                           # 1773 "C:\Program Files (x86)\Microchip\xc8\v1.12\include\pic16f877a.h"
   653                           SSPADD equ 093h ;# 
   654                           # 1779 "C:\Program Files (x86)\Microchip\xc8\v1.12\include\pic16f877a.h"
   655                           SSPSTAT equ 094h ;# 
   656                           # 1947 "C:\Program Files (x86)\Microchip\xc8\v1.12\include\pic16f877a.h"
   657                           TXSTA equ 098h ;# 
   658                           # 2027 "C:\Program Files (x86)\Microchip\xc8\v1.12\include\pic16f877a.h"
   659                           SPBRG equ 099h ;# 
   660                           # 2033 "C:\Program Files (x86)\Microchip\xc8\v1.12\include\pic16f877a.h"
   661                           CMCON equ 09Ch ;# 
   662                           # 2102 "C:\Program Files (x86)\Microchip\xc8\v1.12\include\pic16f877a.h"
   663                           CVRCON equ 09Dh ;# 
   664                           # 2166 "C:\Program Files (x86)\Microchip\xc8\v1.12\include\pic16f877a.h"
   665                           ADRESL equ 09Eh ;# 
   666                           # 2172 "C:\Program Files (x86)\Microchip\xc8\v1.12\include\pic16f877a.h"
   667                           ADCON1 equ 09Fh ;# 
   668                           # 2230 "C:\Program Files (x86)\Microchip\xc8\v1.12\include\pic16f877a.h"
   669                           EEDATA equ 010Ch ;# 
   670                           # 2236 "C:\Program Files (x86)\Microchip\xc8\v1.12\include\pic16f877a.h"
   671                           EEADR equ 010Dh ;# 
   672                           # 2242 "C:\Program Files (x86)\Microchip\xc8\v1.12\include\pic16f877a.h"
   673                           EEDATH equ 010Eh ;# 
   674                           # 2248 "C:\Program Files (x86)\Microchip\xc8\v1.12\include\pic16f877a.h"
   675                           EEADRH equ 010Fh ;# 
   676                           # 2254 "C:\Program Files (x86)\Microchip\xc8\v1.12\include\pic16f877a.h"
   677                           EECON1 equ 018Ch ;# 
   678                           # 2298 "C:\Program Files (x86)\Microchip\xc8\v1.12\include\pic16f877a.h"
   679                           EECON2 equ 018Dh ;# 
   680                           # 46 "C:\Program Files (x86)\Microchip\xc8\v1.12\include\pic16f877a.h"
   681                           INDF equ 00h ;# 
   682                           # 52 "C:\Program Files (x86)\Microchip\xc8\v1.12\include\pic16f877a.h"
   683                           TMR0 equ 01h ;# 
   684                           # 58 "C:\Program Files (x86)\Microchip\xc8\v1.12\include\pic16f877a.h"
   685                           PCL equ 02h ;# 
   686                           # 64 "C:\Program Files (x86)\Microchip\xc8\v1.12\include\pic16f877a.h"
   687                           STATUS equ 03h ;# 
   688                           # 151 "C:\Program Files (x86)\Microchip\xc8\v1.12\include\pic16f877a.h"
   689                           FSR equ 04h ;# 
   690                           # 157 "C:\Program Files (x86)\Microchip\xc8\v1.12\include\pic16f877a.h"
   691                           PORTA equ 05h ;# 
   692                           # 206 "C:\Program Files (x86)\Microchip\xc8\v1.12\include\pic16f877a.h"
   693                           PORTB equ 06h ;# 
   694                           # 267 "C:\Program Files (x86)\Microchip\xc8\v1.12\include\pic16f877a.h"
   695                           PORTC equ 07h ;# 
   696                           # 328 "C:\Program Files (x86)\Microchip\xc8\v1.12\include\pic16f877a.h"
   697                           PORTD equ 08h ;# 
   698                           # 389 "C:\Program Files (x86)\Microchip\xc8\v1.12\include\pic16f877a.h"
   699                           PORTE equ 09h ;# 
   700                           # 420 "C:\Program Files (x86)\Microchip\xc8\v1.12\include\pic16f877a.h"
   701                           PCLATH equ 0Ah ;# 
   702                           # 439 "C:\Program Files (x86)\Microchip\xc8\v1.12\include\pic16f877a.h"
   703                           INTCON equ 0Bh ;# 
   704                           # 516 "C:\Program Files (x86)\Microchip\xc8\v1.12\include\pic16f877a.h"
   705                           PIR1 equ 0Ch ;# 
   706                           # 577 "C:\Program Files (x86)\Microchip\xc8\v1.12\include\pic16f877a.h"
   707                           PIR2 equ 0Dh ;# 
   708                           # 616 "C:\Program Files (x86)\Microchip\xc8\v1.12\include\pic16f877a.h"
   709                           TMR1 equ 0Eh ;# 
   710                           # 622 "C:\Program Files (x86)\Microchip\xc8\v1.12\include\pic16f877a.h"
   711                           TMR1L equ 0Eh ;# 
   712                           # 628 "C:\Program Files (x86)\Microchip\xc8\v1.12\include\pic16f877a.h"
   713                           TMR1H equ 0Fh ;# 
   714                           # 634 "C:\Program Files (x86)\Microchip\xc8\v1.12\include\pic16f877a.h"
   715                           T1CON equ 010h ;# 
   716                           # 708 "C:\Program Files (x86)\Microchip\xc8\v1.12\include\pic16f877a.h"
   717                           TMR2 equ 011h ;# 
   718                           # 714 "C:\Program Files (x86)\Microchip\xc8\v1.12\include\pic16f877a.h"
   719                           T2CON equ 012h ;# 
   720                           # 784 "C:\Program Files (x86)\Microchip\xc8\v1.12\include\pic16f877a.h"
   721                           SSPBUF equ 013h ;# 
   722  0664                     __pmaintext:	;psect for function _main
   723                           opt subtitle "HI-TECH Software Omniscient Code Generator (Lite mode) build 49521"
   724                           
   725                           opt pagewidth 120
   726                           
   727  0038                     	__size_of_main	equ	__end_of_main-_main
   728                           opt subtitle "HI-TECH Software Omniscient Code Generator (Lite mode) build 49521"
   729  0664                     _main:	
   730                           opt subtitle "HI-TECH Software Omniscient Code Generator (Lite mode) build 49521"
   731                           
   732                           opt pagewidth 120
   733                           
   734  0664                     l1047:	
   735                           opt subtitle "HI-TECH Software Omniscient Code Generator (Lite mode) build 49521"
   736  0664  3047               	movlw	(main@test)&0ffh
   737  0665  0084               	movwf	fsr0
   738  0666  3056               	movlw	low(main@F1287)
   739  0667  1283               	bcf	status, 5	;RP0=0, select bank0
   740  0668  1303               	bcf	status, 6	;RP1=0, select bank0
   741  0669  00C3               	movwf	(??_main+0)+0
   742  066A  0804               	movf	fsr0,w
   743  066B  00C4               	movwf	((??_main+0)+0+1)
   744  066C  300F               	movlw	15
   745  066D  00C5               	movwf	((??_main+0)+0+2)
   746  066E                     u340:
   747  066E  0843               	movf	(??_main+0)+0,w
   748  066F  0084               	movwf	fsr0
   749  0670  1383               	bcf	status, 7	;select IRP bank0
   750                           opt subtitle "HI-TECH Software Omniscient Code Generator (Lite mode) build 49521"
   751  0671  0800               	movf	indf,w
   752  0672  00C6               	movwf	((??_main+0)+0+3)
   753  0673  0AC3               	incf	(??_main+0)+0,f
   754  0674  0844               	movf	((??_main+0)+0+1),w
   755  0675  0084               	movwf	fsr0
   756                           opt subtitle "HI-TECH Software Omniscient Code Generator (Lite mode) build 49521"
   757  0676  0846               	movf	((??_main+0)+0+3),w
   758  0677  0080               	movwf	indf
   759  0678  0AC4               	incf	((??_main+0)+0+1),f
   760  0679  0BC5               	decfsz	((??_main+0)+0+2),f
   761  067A  2E6E               	goto	u340
   762                           opt subtitle "HI-TECH Software Omniscient Code Generator (Lite mode) build 49521"
   763                           
   764  067B                     l1049:	
   765                           opt subtitle "HI-TECH Software Omniscient Code Generator (Lite mode) build 49521"
   766  067B  120A  118A  2729   	fcall	_api_lcd_initialize
              120A  118A         
   767                           opt subtitle "HI-TECH Software Omniscient Code Generator (Lite mode) build 49521"
   768                           
   769  0680                     l1051:	
   770                           opt subtitle "HI-TECH Software Omniscient Code Generator (Lite mode) build 49521"
   771  0680  3001               	movlw	(01h)
   772  0681  120A  118A  25F1   	fcall	_api_lcd_backlight
              120A  118A         
   773                           opt subtitle "HI-TECH Software Omniscient Code Generator (Lite mode) build 49521"
   774                           
   775  0686                     l1053:	
   776                           opt subtitle "HI-TECH Software Omniscient Code Generator (Lite mode) build 49521"
   777  0686  01F7               	clrf	(?_api_lcd_printf)
   778  0687  0AF7               	incf	(?_api_lcd_printf),f
   779  0688  3047               	movlw	(main@test)&0ffh
   780  0689  1283               	bcf	status, 5	;RP0=0, select bank0
   781  068A  1303               	bcf	status, 6	;RP1=0, select bank0
   782  068B  00C3               	movwf	(??_main+0)+0
   783  068C  0843               	movf	(??_main+0)+0,w
   784  068D  00F8               	movwf	0+(?_api_lcd_printf)+01h
   785  068E  300E               	movlw	(0Eh)
   786  068F  00C4               	movwf	(??_main+1)+0
   787  0690  0844               	movf	(??_main+1)+0,w
   788  0691  00F9               	movwf	0+(?_api_lcd_printf)+02h
   789  0692  3001               	movlw	(01h)
   790  0693  120A  118A  2783   	fcall	_api_lcd_printf
              120A  118A         
   791                           opt subtitle "HI-TECH Software Omniscient Code Generator (Lite mode) build 49521"
   792                           
   793                           opt pagewidth 120
   794  0698                     l118:	
   795                           opt subtitle "HI-TECH Software Omniscient Code Generator (Lite mode) build 49521"
   796  0698                     l119:	
   797  0698  2E98               	goto	l118
   798                           opt subtitle "HI-TECH Software Omniscient Code Generator (Lite mode) build 49521"
   799  0699                     l120:	
   800                           opt subtitle "HI-TECH Software Omniscient Code Generator (Lite mode) build 49521"
   801                           
   802                           opt pagewidth 120
   803                           
   804  0699                     l121:	
   805                           opt subtitle "HI-TECH Software Omniscient Code Generator (Lite mode) build 49521"
   806  0699  120A  118A  2800   	ljmp	start
   807                           opt subtitle "HI-TECH Software Omniscient Code Generator (Lite mode) build 49521"
   808                           
   809  069C                     	__end_of_main:
   810                           opt subtitle "HI-TECH Software Omniscient Code Generator (Lite mode) build 49521"
   811                           
   812                           opt pagewidth 120
   813                           
   814                           	opt lm
   815                           
   816                           	processor	16F877A
   817                           clrc	macro
   818                           	bcf	3,0
   819                           	endm
   820                           clrz	macro
   821                           	bcf	3,2
   822                           	endm
   823                           setc	macro
   824                           	bsf	3,0
   825                           	endm
   826                           setz	macro
   827                           	bsf	3,2
   828                           	endm
   829                           skipc	macro
   830                           	btfss	3,0
   831                           	endm
   832                           skipz	macro
   833                           	btfss	3,2
   834                           	endm
   835                           skipnc	macro
   836                           	btfsc	3,0
   837                           	endm
   838                           skipnz	macro
   839                           	btfsc	3,2
   840                           	endm
   841                           indf	equ	0
   842                           indf0	equ	0
   843                           pc	equ	2
   844                           pcl	equ	2
   845                           status	equ	3
   846                           fsr	equ	4
   847                           fsr0	equ	4
   848  0729                     __ptext263:	;psect for function _api_lcd_initialize
   849                           opt subtitle "HI-TECH Software Omniscient Code Generator (Lite mode) build 49521"
   850                           
   851                           opt pagewidth 120
   852                           
   853  005A                     	__size_of_api_lcd_initialize	equ	__end_of_api_lcd_initialize-_api_lcd_initialize
   854                           opt subtitle "HI-TECH Software Omniscient Code Generator (Lite mode) build 49521"
   855  0729                     _api_lcd_initialize:	
   856                           opt subtitle "HI-TECH Software Omniscient Code Generator (Lite mode) build 49521"
   857                           
   858                           opt pagewidth 120
   859                           
   860  0729                     l929:	
   861                           opt subtitle "HI-TECH Software Omniscient Code Generator (Lite mode) build 49521"
   862  0729  1683               	bsf	status, 5	;RP0=1, select bank1
   863  072A  1303               	bcf	status, 6	;RP1=0, select bank1
   864  072B  1006               	bcf	(134)^080h,0	;volatile
   865                           opt subtitle "HI-TECH Software Omniscient Code Generator (Lite mode) build 49521"
   866                           
   867  072C  1086               	bcf	(134)^080h,1	;volatile
   868                           opt subtitle "HI-TECH Software Omniscient Code Generator (Lite mode) build 49521"
   869                           
   870  072D  1106               	bcf	(134)^080h,2	;volatile
   871                           opt subtitle "HI-TECH Software Omniscient Code Generator (Lite mode) build 49521"
   872                           
   873  072E  1186               	bcf	(134)^080h,3	;volatile
   874                           opt subtitle "HI-TECH Software Omniscient Code Generator (Lite mode) build 49521"
   875                           
   876  072F                     l931:	
   877                           opt subtitle "HI-TECH Software Omniscient Code Generator (Lite mode) build 49521"
   878  072F  0188               	clrf	(136)^080h	;volatile
   879                           opt subtitle "HI-TECH Software Omniscient Code Generator (Lite mode) build 49521"
   880                           
   881  0730                     l933:	
   882                           opt subtitle "HI-TECH Software Omniscient Code Generator (Lite mode) build 49521"
   883  0730  1283               	bcf	status, 5	;RP0=0, select bank0
   884  0731  1303               	bcf	status, 6	;RP1=0, select bank0
   885  0732  1006               	bcf	(6),0	;volatile
   886                           opt subtitle "HI-TECH Software Omniscient Code Generator (Lite mode) build 49521"
   887                           
   888  0733                     l935:	
   889                           opt subtitle "HI-TECH Software Omniscient Code Generator (Lite mode) build 49521"
   890  0733  1086               	bcf	(6),1	;volatile
   891                           opt subtitle "HI-TECH Software Omniscient Code Generator (Lite mode) build 49521"
   892                           
   893  0734                     l937:	
   894                           opt subtitle "HI-TECH Software Omniscient Code Generator (Lite mode) build 49521"
   895  0734  1106               	bcf	(6),2	;volatile
   896                           opt subtitle "HI-TECH Software Omniscient Code Generator (Lite mode) build 49521"
   897                           
   898  0735                     l939:	
   899                           opt subtitle "HI-TECH Software Omniscient Code Generator (Lite mode) build 49521"
   900  0735  1186               	bcf	(6),3	;volatile
   901                           opt subtitle "HI-TECH Software Omniscient Code Generator (Lite mode) build 49521"
   902                           
   903  0736  0188               	clrf	(8)	;volatile
   904                           opt subtitle "HI-TECH Software Omniscient Code Generator (Lite mode) build 49521"
   905                           
   906  0737                     l941:	
   907                           opt subtitle "HI-TECH Software Omniscient Code Generator (Lite mode) build 49521"
   908  0737  120A  118A  25A8   	fcall	_lcd_cmd
              120A  118A         
   909                           opt subtitle "HI-TECH Software Omniscient Code Generator (Lite mode) build 49521"
   910                           
   911  073C                     l943:	
   912                           opt subtitle "HI-TECH Software Omniscient Code Generator (Lite mode) build 49521"
   913  073C  3001               	movlw	(01h)
   914  073D  120A  118A  25DC   	fcall	_lcd_rw
              120A  118A         
   915                           opt subtitle "HI-TECH Software Omniscient Code Generator (Lite mode) build 49521"
   916                           
   917  0742                     l945:	
   918                           opt subtitle "HI-TECH Software Omniscient Code Generator (Lite mode) build 49521"
   919  0742  3038               	movlw	(038h)
   920  0743  120A  118A  25AC   	fcall	_lcd_write
              120A  118A         
   921                           opt subtitle "HI-TECH Software Omniscient Code Generator (Lite mode) build 49521"
   922                           
   923  0748                     l947:	
   924                           opt subtitle "HI-TECH Software Omniscient Code Generator (Lite mode) build 49521"
   925  0748  120A  118A  2606   	fcall	_lcd_en
              120A  118A         
   926                           opt subtitle "HI-TECH Software Omniscient Code Generator (Lite mode) build 49521"
   927                           
   928  074D                     l949:	
   929                           opt subtitle "HI-TECH Software Omniscient Code Generator (Lite mode) build 49521"
   930  074D  120A  118A  2606   	fcall	_lcd_en
              120A  118A         
   931                           opt subtitle "HI-TECH Software Omniscient Code Generator (Lite mode) build 49521"
   932                           
   933  0752                     l951:	
   934                           opt subtitle "HI-TECH Software Omniscient Code Generator (Lite mode) build 49521"
   935  0752  120A  118A  2606   	fcall	_lcd_en
              120A  118A         
   936                           opt subtitle "HI-TECH Software Omniscient Code Generator (Lite mode) build 49521"
   937                           
   938  0757                     l953:	
   939                           opt subtitle "HI-TECH Software Omniscient Code Generator (Lite mode) build 49521"
   940  0757  120A  118A  2606   	fcall	_lcd_en
              120A  118A         
   941                           opt subtitle "HI-TECH Software Omniscient Code Generator (Lite mode) build 49521"
   942                           
   943  075C                     l955:	
   944                           opt subtitle "HI-TECH Software Omniscient Code Generator (Lite mode) build 49521"
   945  075C  300C               	movlw	(0Ch)
   946  075D  120A  118A  25AC   	fcall	_lcd_write
              120A  118A         
   947                           opt subtitle "HI-TECH Software Omniscient Code Generator (Lite mode) build 49521"
   948                           
   949  0762                     l957:	
   950                           opt subtitle "HI-TECH Software Omniscient Code Generator (Lite mode) build 49521"
   951  0762  120A  118A  2606   	fcall	_lcd_en
              120A  118A         
   952                           opt subtitle "HI-TECH Software Omniscient Code Generator (Lite mode) build 49521"
   953                           
   954  0767                     l959:	
   955                           opt subtitle "HI-TECH Software Omniscient Code Generator (Lite mode) build 49521"
   956  0767  3080               	movlw	(080h)
   957  0768  120A  118A  25AC   	fcall	_lcd_write
              120A  118A         
   958                           opt subtitle "HI-TECH Software Omniscient Code Generator (Lite mode) build 49521"
   959                           
   960  076D                     l961:	
   961                           opt subtitle "HI-TECH Software Omniscient Code Generator (Lite mode) build 49521"
   962  076D  120A  118A  2606   	fcall	_lcd_en
              120A  118A         
   963                           opt subtitle "HI-TECH Software Omniscient Code Generator (Lite mode) build 49521"
   964                           
   965  0772                     l963:	
   966                           opt subtitle "HI-TECH Software Omniscient Code Generator (Lite mode) build 49521"
   967  0772  3001               	movlw	(01h)
   968  0773  120A  118A  25AC   	fcall	_lcd_write
              120A  118A         
   969                           opt subtitle "HI-TECH Software Omniscient Code Generator (Lite mode) build 49521"
   970                           
   971  0778                     l965:	
   972                           opt subtitle "HI-TECH Software Omniscient Code Generator (Lite mode) build 49521"
   973  0778  120A  118A  2606   	fcall	_lcd_en
              120A  118A         
   974                           opt subtitle "HI-TECH Software Omniscient Code Generator (Lite mode) build 49521"
   975                           
   976  077D                     l967:	
   977                           opt subtitle "HI-TECH Software Omniscient Code Generator (Lite mode) build 49521"
   978  077D  120A  118A  25A4   	fcall	_lcd_data
              120A  118A         
   979                           opt subtitle "HI-TECH Software Omniscient Code Generator (Lite mode) build 49521"
   980                           
   981  0782                     l27:	
   982  0782  0008               	return
   983                           opt subtitle "HI-TECH Software Omniscient Code Generator (Lite mode) build 49521"
   984                           
   985  0783                     	__end_of_api_lcd_initialize:
   986                           opt subtitle "HI-TECH Software Omniscient Code Generator (Lite mode) build 49521"
   987                           
   988                           opt pagewidth 120
   989                           
   990                           	opt lm
   991                           
   992                           	processor	16F877A
   993                           clrc	macro
   994                           	bcf	3,0
   995                           	endm
   996                           clrz	macro
   997                           	bcf	3,2
   998                           	endm
   999                           setc	macro
  1000                           	bsf	3,0
  1001                           	endm
  1002                           setz	macro
  1003                           	bsf	3,2
  1004                           	endm
  1005                           skipc	macro
  1006                           	btfss	3,0
  1007                           	endm
  1008                           skipz	macro
  1009                           	btfss	3,2
  1010                           	endm
  1011                           skipnc	macro
  1012                           	btfsc	3,0
  1013                           	endm
  1014                           skipnz	macro
  1015                           	btfsc	3,2
  1016                           	endm
  1017                           indf	equ	0
  1018                           indf0	equ	0
  1019  05F1                     __ptext264:	;psect for function _api_lcd_backlight
  1020                           opt subtitle "HI-TECH Software Omniscient Code Generator (Lite mode) build 49521"
  1021                           
  1022                           opt pagewidth 120
  1023                           
  1024  0015                     	__size_of_api_lcd_backlight	equ	__end_of_api_lcd_backlight-_api_lcd_backlight
  1025                           opt subtitle "HI-TECH Software Omniscient Code Generator (Lite mode) build 49521"
  1026  05F1                     _api_lcd_backlight:	
  1027                           opt subtitle "HI-TECH Software Omniscient Code Generator (Lite mode) build 49521"
  1028                           
  1029                           opt pagewidth 120
  1030  05F1  00F0               	movwf	(api_lcd_backlight@state)
  1031                           opt subtitle "HI-TECH Software Omniscient Code Generator (Lite mode) build 49521"
  1032                           
  1033  05F2                     l835:	
  1034                           opt subtitle "HI-TECH Software Omniscient Code Generator (Lite mode) build 49521"
  1035  05F2  2DFD               	goto	l839
  1036                           opt subtitle "HI-TECH Software Omniscient Code Generator (Lite mode) build 49521"
  1037                           
  1038                           opt pagewidth 120
  1039                           
  1040  05F3                     l31:	
  1041  05F3  1283               	bcf	status, 5	;RP0=0, select bank0
  1042  05F4  1303               	bcf	status, 6	;RP1=0, select bank0
  1043  05F5  1186               	bcf	(6),3	;volatile
  1044  05F6  2E05               	goto	l35
  1045                           opt subtitle "HI-TECH Software Omniscient Code Generator (Lite mode) build 49521"
  1046                           
  1047                           opt pagewidth 120
  1048  05F7                     l33:	
  1049  05F7  1283               	bcf	status, 5	;RP0=0, select bank0
  1050  05F8  1303               	bcf	status, 6	;RP1=0, select bank0
  1051  05F9  1586               	bsf	(6),3	;volatile
  1052  05FA  2E05               	goto	l35
  1053                           opt subtitle "HI-TECH Software Omniscient Code Generator (Lite mode) build 49521"
  1054                           
  1055                           opt pagewidth 120
  1056  05FB                     l34:	
  1057  05FB  2E05               	goto	l35
  1058                           opt subtitle "HI-TECH Software Omniscient Code Generator (Lite mode) build 49521"
  1059                           
  1060  05FC                     l837:	
  1061                           opt subtitle "HI-TECH Software Omniscient Code Generator (Lite mode) build 49521"
  1062  05FC  2E05               	goto	l35
  1063                           opt subtitle "HI-TECH Software Omniscient Code Generator (Lite mode) build 49521"
  1064                           
  1065  05FD                     l30:	
  1066                           opt subtitle "HI-TECH Software Omniscient Code Generator (Lite mode) build 49521"
  1067  05FD                     l839:	
  1068  05FD  0870               	movf	(api_lcd_backlight@state),w
  1069                           opt subtitle "HI-TECH Software Omniscient Code Generator (Lite mode) build 49521"
  1070                           
  1071                           opt pagewidth 120
  1072                           
  1073                           	opt lm
  1074                           
  1075                           	processor	16F877A
  1076                           clrc	macro
  1077                           	bcf	3,0
  1078                           	endm
  1079                           clrz	macro
  1080                           	bcf	3,2
  1081                           	endm
  1082  05FE  3A00               	xorlw	0^0	; case 0
  1083  05FF  1903               	skipnz
  1084  0600  2DF3               	goto	l31
  1085  0601  3A01               	xorlw	1^0	; case 1
  1086  0602  1903               	skipnz
  1087  0603  2DF7               	goto	l33
  1088  0604  2E05               	goto	l35
  1089                           opt subtitle "HI-TECH Software Omniscient Code Generator (Lite mode) build 49521"
  1090                           
  1091                           opt pagewidth 120
  1092                           
  1093  0605                     l32:	
  1094                           opt subtitle "HI-TECH Software Omniscient Code Generator (Lite mode) build 49521"
  1095                           
  1096  0605                     l35:	
  1097  0605  0008               	return
  1098                           opt subtitle "HI-TECH Software Omniscient Code Generator (Lite mode) build 49521"
  1099                           
  1100  0606                     	__end_of_api_lcd_backlight:
  1101                           opt subtitle "HI-TECH Software Omniscient Code Generator (Lite mode) build 49521"
  1102                           
  1103                           opt pagewidth 120
  1104                           
  1105                           	opt lm
  1106                           
  1107                           	processor	16F877A
  1108                           clrc	macro
  1109                           	bcf	3,0
  1110                           	endm
  1111                           clrz	macro
  1112                           	bcf	3,2
  1113                           	endm
  1114                           setc	macro
  1115                           	bsf	3,0
  1116                           	endm
  1117                           setz	macro
  1118                           	bsf	3,2
  1119                           	endm
  1120                           skipc	macro
  1121                           	btfss	3,0
  1122                           	endm
  1123                           skipz	macro
  1124                           	btfss	3,2
  1125                           	endm
  1126                           skipnc	macro
  1127                           	btfsc	3,0
  1128                           	endm
  1129                           skipnz	macro
  1130                           	btfsc	3,2
  1131                           	endm
  1132                           indf	equ	0
  1133                           indf0	equ	0
  1134                           pc	equ	2
  1135                           pcl	equ	2
  1136                           status	equ	3
  1137                           fsr	equ	4
  1138                           fsr0	equ	4
  1139                           c	equ	1
  1140                           z	equ	0
  1141  0783                     __ptext265:	;psect for function _api_lcd_printf
  1142                           opt subtitle "HI-TECH Software Omniscient Code Generator (Lite mode) build 49521"
  1143                           
  1144                           opt pagewidth 120
  1145                           
  1146  007D                     	__size_of_api_lcd_printf	equ	__end_of_api_lcd_printf-_api_lcd_printf
  1147                           opt subtitle "HI-TECH Software Omniscient Code Generator (Lite mode) build 49521"
  1148  0783                     _api_lcd_printf:	
  1149                           opt subtitle "HI-TECH Software Omniscient Code Generator (Lite mode) build 49521"
  1150                           
  1151                           opt pagewidth 120
  1152  0783  1283               	bcf	status, 5	;RP0=0, select bank0
  1153  0784  1303               	bcf	status, 6	;RP1=0, select bank0
  1154  0785  00C0               	movwf	(api_lcd_printf@line)
  1155                           opt subtitle "HI-TECH Software Omniscient Code Generator (Lite mode) build 49521"
  1156                           
  1157  0786                     l1021:	
  1158                           opt subtitle "HI-TECH Software Omniscient Code Generator (Lite mode) build 49521"
  1159  0786  01C1               	clrf	(api_lcd_printf@i)
  1160  0787  01C2               	clrf	(api_lcd_printf@j)
  1161                           opt subtitle "HI-TECH Software Omniscient Code Generator (Lite mode) build 49521"
  1162                           
  1163  0788                     l1023:	
  1164                           opt subtitle "HI-TECH Software Omniscient Code Generator (Lite mode) build 49521"
  1165  0788  0877               	movf	(api_lcd_printf@cursor),w
  1166  0789  3EFF               	addlw	0FFh
  1167  078A  00FA               	movwf	(??_api_lcd_printf+0)+0
  1168  078B  087A               	movf	(??_api_lcd_printf+0)+0,w
  1169  078C  00C1               	movwf	(api_lcd_printf@i)
  1170                           opt subtitle "HI-TECH Software Omniscient Code Generator (Lite mode) build 49521"
  1171                           
  1172  078D  2FF0               	goto	l1043
  1173                           opt subtitle "HI-TECH Software Omniscient Code Generator (Lite mode) build 49521"
  1174                           
  1175                           opt pagewidth 120
  1176                           
  1177  078E                     l79:	
  1178                           opt subtitle "HI-TECH Software Omniscient Code Generator (Lite mode) build 49521"
  1179                           
  1180                           opt pagewidth 120
  1181  078E  2FA7               	goto	l1031
  1182                           opt subtitle "HI-TECH Software Omniscient Code Generator (Lite mode) build 49521"
  1183  078F                     l81:	
  1184                           opt subtitle "HI-TECH Software Omniscient Code Generator (Lite mode) build 49521"
  1185                           
  1186  078F                     l1025:	
  1187                           opt subtitle "HI-TECH Software Omniscient Code Generator (Lite mode) build 49521"
  1188                           
  1189  078F  1283               	bcf	status, 5	;RP0=0, select bank0
  1190  0790  1303               	bcf	status, 6	;RP1=0, select bank0
  1191  0791  0842               	movf	(api_lcd_printf@j),w
  1192  0792  0778               	addwf	(api_lcd_printf@databuffer),w
  1193  0793  00FA               	movwf	(??_api_lcd_printf+0)+0
  1194  0794  087A               	movf	0+(??_api_lcd_printf+0)+0,w
  1195  0795  0084               	movwf	fsr0
  1196  0796  1383               	bcf	status, 7	;select IRP bank0
  1197  0797  0800               	movf	indf,w
  1198  0798  00FB               	movwf	(??_api_lcd_printf+1)+0
  1199  0799  0841               	movf	(api_lcd_printf@i),w
  1200  079A  3E20               	addlw	_lcd_buffer_1&0ffh
  1201  079B  0084               	movwf	fsr0
  1202  079C  087B               	movf	(??_api_lcd_printf+1)+0,w
  1203  079D  0080               	movwf	indf
  1204                           opt subtitle "HI-TECH Software Omniscient Code Generator (Lite mode) build 49521"
  1205                           
  1206  079E                     l1027:	
  1207                           opt subtitle "HI-TECH Software Omniscient Code Generator (Lite mode) build 49521"
  1208  079E  3001               	movlw	(01h)
  1209  079F  00FA               	movwf	(??_api_lcd_printf+0)+0
  1210  07A0  087A               	movf	(??_api_lcd_printf+0)+0,w
  1211  07A1  07C2               	addwf	(api_lcd_printf@j),f
  1212                           opt subtitle "HI-TECH Software Omniscient Code Generator (Lite mode) build 49521"
  1213                           
  1214  07A2                     l1029:	
  1215                           opt subtitle "HI-TECH Software Omniscient Code Generator (Lite mode) build 49521"
  1216  07A2  3001               	movlw	(01h)
  1217  07A3  00FA               	movwf	(??_api_lcd_printf+0)+0
  1218  07A4  087A               	movf	(??_api_lcd_printf+0)+0,w
  1219  07A5  07C1               	addwf	(api_lcd_printf@i),f
  1220  07A6  2FA7               	goto	l1031
  1221                           opt subtitle "HI-TECH Software Omniscient Code Generator (Lite mode) build 49521"
  1222                           
  1223  07A7                     l80:	
  1224                           opt subtitle "HI-TECH Software Omniscient Code Generator (Lite mode) build 49521"
  1225                           
  1226  07A7                     l1031:	
  1227  07A7  0879               	movf	(api_lcd_printf@data_length),w
  1228  07A8  3EFF               	addlw	low(-1)
  1229  07A9  00FA               	movwf	(??_api_lcd_printf+0)+0
  1230  07AA  30FF               	movlw	high(-1)
  1231  07AB  1803               	skipnc
  1232  07AC  3000               	movlw	(high(-1)+1)&0ffh
  1233  07AD  00FB               	movwf	((??_api_lcd_printf+0)+0)+1
  1234  07AE  087B               	movf	1+(??_api_lcd_printf+0)+0,w
  1235  07AF  3A80               	xorlw	80h
  1236  07B0  00FC               	movwf	(??_api_lcd_printf+2)+0
  1237  07B1  3080               	movlw	80h
  1238  07B2  027C               	subwf	(??_api_lcd_printf+2)+0,w
  1239  07B3  1D03               	skipz
  1240  07B4  2FB7               	goto	u325
  1241  07B5  0842               	movf	(api_lcd_printf@j),w
  1242  07B6  027A               	subwf	0+(??_api_lcd_printf+0)+0,w
  1243  07B7                     u325:
  1244                           opt subtitle "HI-TECH Software Omniscient Code Generator (Lite mode) build 49521"
  1245  07B7  1803               	skipnc
  1246  07B8  2FBA               	goto	u321
  1247  07B9  2FBB               	goto	u320
  1248  07BA                     u321:
  1249  07BA  2F8F               	goto	l1025
  1250  07BB                     u320:
  1251  07BB  2FFA               	goto	l1045
  1252                           opt subtitle "HI-TECH Software Omniscient Code Generator (Lite mode) build 49521"
  1253  07BC                     l82:	
  1254                           opt subtitle "HI-TECH Software Omniscient Code Generator (Lite mode) build 49521"
  1255                           
  1256                           opt pagewidth 120
  1257  07BC  2FFA               	goto	l1045
  1258                           opt subtitle "HI-TECH Software Omniscient Code Generator (Lite mode) build 49521"
  1259                           
  1260                           opt pagewidth 120
  1261  07BD                     l84:	
  1262                           opt subtitle "HI-TECH Software Omniscient Code Generator (Lite mode) build 49521"
  1263                           
  1264                           opt pagewidth 120
  1265  07BD  2FD6               	goto	l1039
  1266                           opt subtitle "HI-TECH Software Omniscient Code Generator (Lite mode) build 49521"
  1267  07BE                     l86:	
  1268                           opt subtitle "HI-TECH Software Omniscient Code Generator (Lite mode) build 49521"
  1269                           
  1270  07BE                     l1033:	
  1271                           opt subtitle "HI-TECH Software Omniscient Code Generator (Lite mode) build 49521"
  1272                           
  1273  07BE  1283               	bcf	status, 5	;RP0=0, select bank0
  1274  07BF  1303               	bcf	status, 6	;RP1=0, select bank0
  1275  07C0  0842               	movf	(api_lcd_printf@j),w
  1276  07C1  0778               	addwf	(api_lcd_printf@databuffer),w
  1277  07C2  00FA               	movwf	(??_api_lcd_printf+0)+0
  1278  07C3  087A               	movf	0+(??_api_lcd_printf+0)+0,w
  1279  07C4  0084               	movwf	fsr0
  1280  07C5  1383               	bcf	status, 7	;select IRP bank0
  1281  07C6  0800               	movf	indf,w
  1282  07C7  00FB               	movwf	(??_api_lcd_printf+1)+0
  1283  07C8  0841               	movf	(api_lcd_printf@i),w
  1284  07C9  3E30               	addlw	_lcd_buffer_2&0ffh
  1285  07CA  0084               	movwf	fsr0
  1286  07CB  087B               	movf	(??_api_lcd_printf+1)+0,w
  1287  07CC  0080               	movwf	indf
  1288                           opt subtitle "HI-TECH Software Omniscient Code Generator (Lite mode) build 49521"
  1289                           
  1290  07CD                     l1035:	
  1291                           opt subtitle "HI-TECH Software Omniscient Code Generator (Lite mode) build 49521"
  1292  07CD  3001               	movlw	(01h)
  1293  07CE  00FA               	movwf	(??_api_lcd_printf+0)+0
  1294  07CF  087A               	movf	(??_api_lcd_printf+0)+0,w
  1295  07D0  07C2               	addwf	(api_lcd_printf@j),f
  1296                           opt subtitle "HI-TECH Software Omniscient Code Generator (Lite mode) build 49521"
  1297                           
  1298  07D1                     l1037:	
  1299                           opt subtitle "HI-TECH Software Omniscient Code Generator (Lite mode) build 49521"
  1300  07D1  3001               	movlw	(01h)
  1301  07D2  00FA               	movwf	(??_api_lcd_printf+0)+0
  1302  07D3  087A               	movf	(??_api_lcd_printf+0)+0,w
  1303  07D4  07C1               	addwf	(api_lcd_printf@i),f
  1304  07D5  2FD6               	goto	l1039
  1305                           opt subtitle "HI-TECH Software Omniscient Code Generator (Lite mode) build 49521"
  1306                           
  1307  07D6                     l85:	
  1308                           opt subtitle "HI-TECH Software Omniscient Code Generator (Lite mode) build 49521"
  1309                           
  1310  07D6                     l1039:	
  1311  07D6  0879               	movf	(api_lcd_printf@data_length),w
  1312  07D7  3EFF               	addlw	low(-1)
  1313  07D8  00FA               	movwf	(??_api_lcd_printf+0)+0
  1314  07D9  30FF               	movlw	high(-1)
  1315  07DA  1803               	skipnc
  1316  07DB  3000               	movlw	(high(-1)+1)&0ffh
  1317  07DC  00FB               	movwf	((??_api_lcd_printf+0)+0)+1
  1318  07DD  087B               	movf	1+(??_api_lcd_printf+0)+0,w
  1319  07DE  3A80               	xorlw	80h
  1320  07DF  00FC               	movwf	(??_api_lcd_printf+2)+0
  1321  07E0  3080               	movlw	80h
  1322  07E1  027C               	subwf	(??_api_lcd_printf+2)+0,w
  1323  07E2  1D03               	skipz
  1324  07E3  2FE8               	goto	u335
  1325  07E4  1283               	bcf	status, 5	;RP0=0, select bank0
  1326  07E5  1303               	bcf	status, 6	;RP1=0, select bank0
  1327  07E6  0842               	movf	(api_lcd_printf@j),w
  1328  07E7  027A               	subwf	0+(??_api_lcd_printf+0)+0,w
  1329  07E8                     u335:
  1330                           opt subtitle "HI-TECH Software Omniscient Code Generator (Lite mode) build 49521"
  1331  07E8  1803               	skipnc
  1332  07E9  2FEB               	goto	u331
  1333  07EA  2FEC               	goto	u330
  1334  07EB                     u331:
  1335  07EB  2FBE               	goto	l1033
  1336  07EC                     u330:
  1337  07EC  2FFA               	goto	l1045
  1338                           opt subtitle "HI-TECH Software Omniscient Code Generator (Lite mode) build 49521"
  1339  07ED                     l87:	
  1340                           opt subtitle "HI-TECH Software Omniscient Code Generator (Lite mode) build 49521"
  1341                           
  1342                           opt pagewidth 120
  1343  07ED  2FFA               	goto	l1045
  1344                           opt subtitle "HI-TECH Software Omniscient Code Generator (Lite mode) build 49521"
  1345                           
  1346                           opt pagewidth 120
  1347  07EE                     l88:	
  1348  07EE  2FFA               	goto	l1045
  1349                           opt subtitle "HI-TECH Software Omniscient Code Generator (Lite mode) build 49521"
  1350                           
  1351  07EF                     l1041:	
  1352                           opt subtitle "HI-TECH Software Omniscient Code Generator (Lite mode) build 49521"
  1353  07EF  2FFA               	goto	l1045
  1354                           opt subtitle "HI-TECH Software Omniscient Code Generator (Lite mode) build 49521"
  1355                           
  1356  07F0                     l78:	
  1357                           opt subtitle "HI-TECH Software Omniscient Code Generator (Lite mode) build 49521"
  1358  07F0                     l1043:	
  1359  07F0  1283               	bcf	status, 5	;RP0=0, select bank0
  1360  07F1  1303               	bcf	status, 6	;RP1=0, select bank0
  1361  07F2  0840               	movf	(api_lcd_printf@line),w
  1362                           opt subtitle "HI-TECH Software Omniscient Code Generator (Lite mode) build 49521"
  1363                           
  1364                           opt pagewidth 120
  1365                           
  1366                           	opt lm
  1367                           
  1368                           	processor	16F877A
  1369                           clrc	macro
  1370                           	bcf	3,0
  1371                           	endm
  1372  07F3  3A01               	xorlw	1^0	; case 1
  1373  07F4  1903               	skipnz
  1374  07F5  2FA7               	goto	l1031
  1375  07F6  3A03               	xorlw	2^1	; case 2
  1376  07F7  1903               	skipnz
  1377  07F8  2FD6               	goto	l1039
  1378  07F9  2FFA               	goto	l1045
  1379                           opt subtitle "HI-TECH Software Omniscient Code Generator (Lite mode) build 49521"
  1380                           
  1381                           opt pagewidth 120
  1382                           
  1383  07FA                     l83:	
  1384                           opt subtitle "HI-TECH Software Omniscient Code Generator (Lite mode) build 49521"
  1385                           
  1386  07FA                     l1045:	
  1387                           opt subtitle "HI-TECH Software Omniscient Code Generator (Lite mode) build 49521"
  1388  07FA  120A  118A  26D5   	fcall	_lcd_printf
              120A  118A         
  1389                           opt subtitle "HI-TECH Software Omniscient Code Generator (Lite mode) build 49521"
  1390                           
  1391  07FF                     l89:	
  1392  07FF  0008               	return
  1393                           opt subtitle "HI-TECH Software Omniscient Code Generator (Lite mode) build 49521"
  1394                           
  1395  0800                     	__end_of_api_lcd_printf:
  1396                           opt subtitle "HI-TECH Software Omniscient Code Generator (Lite mode) build 49521"
  1397                           
  1398                           opt pagewidth 120
  1399                           
  1400                           	opt lm
  1401                           
  1402                           	processor	16F877A
  1403                           clrc	macro
  1404                           	bcf	3,0
  1405                           	endm
  1406                           clrz	macro
  1407                           	bcf	3,2
  1408                           	endm
  1409                           setc	macro
  1410                           	bsf	3,0
  1411                           	endm
  1412                           setz	macro
  1413                           	bsf	3,2
  1414                           	endm
  1415                           skipc	macro
  1416                           	btfss	3,0
  1417                           	endm
  1418                           skipz	macro
  1419                           	btfss	3,2
  1420                           	endm
  1421                           skipnc	macro
  1422                           	btfsc	3,0
  1423                           	endm
  1424                           skipnz	macro
  1425                           	btfsc	3,2
  1426                           	endm
  1427                           indf	equ	0
  1428                           indf0	equ	0
  1429                           pc	equ	2
  1430                           pcl	equ	2
  1431                           status	equ	3
  1432                           fsr	equ	4
  1433                           fsr0	equ	4
  1434  06D5                     __ptext266:	;psect for function _lcd_printf
  1435                           opt subtitle "HI-TECH Software Omniscient Code Generator (Lite mode) build 49521"
  1436                           
  1437                           opt pagewidth 120
  1438                           
  1439  0054                     	__size_of_lcd_printf	equ	__end_of_lcd_printf-_lcd_printf
  1440                           opt subtitle "HI-TECH Software Omniscient Code Generator (Lite mode) build 49521"
  1441  06D5                     _lcd_printf:	
  1442                           opt subtitle "HI-TECH Software Omniscient Code Generator (Lite mode) build 49521"
  1443                           
  1444                           opt pagewidth 120
  1445                           
  1446  06D5                     l987:	
  1447                           opt subtitle "HI-TECH Software Omniscient Code Generator (Lite mode) build 49521"
  1448  06D5  01F6               	clrf	(lcd_printf@i)
  1449                           opt subtitle "HI-TECH Software Omniscient Code Generator (Lite mode) build 49521"
  1450                           
  1451  06D6                     l989:	
  1452                           opt subtitle "HI-TECH Software Omniscient Code Generator (Lite mode) build 49521"
  1453  06D6  3001               	movlw	(01h)
  1454  06D7  120A  118A  269C   	fcall	_lcd_set_line
              120A  118A         
  1455                           opt subtitle "HI-TECH Software Omniscient Code Generator (Lite mode) build 49521"
  1456                           
  1457  06DC                     l991:	
  1458                           opt subtitle "HI-TECH Software Omniscient Code Generator (Lite mode) build 49521"
  1459  06DC  01F6               	clrf	(lcd_printf@i)
  1460                           opt subtitle "HI-TECH Software Omniscient Code Generator (Lite mode) build 49521"
  1461  06DD                     l993:	
  1462  06DD  3010               	movlw	(010h)
  1463  06DE  0276               	subwf	(lcd_printf@i),w
  1464  06DF  1C03               	skipc
  1465  06E0  2EE2               	goto	u281
  1466  06E1  2EE3               	goto	u280
  1467  06E2                     u281:
  1468  06E2  2EE5               	goto	l997
  1469  06E3                     u280:
  1470  06E3  2EFF               	goto	l1005
  1471                           opt subtitle "HI-TECH Software Omniscient Code Generator (Lite mode) build 49521"
  1472  06E4                     l995:	
  1473  06E4  2EFF               	goto	l1005
  1474                           opt subtitle "HI-TECH Software Omniscient Code Generator (Lite mode) build 49521"
  1475  06E5                     l66:	
  1476                           opt subtitle "HI-TECH Software Omniscient Code Generator (Lite mode) build 49521"
  1477  06E5                     l997:	
  1478  06E5  0876               	movf	(lcd_printf@i),w
  1479  06E6  3E20               	addlw	_lcd_buffer_1&0ffh
  1480  06E7  0084               	movwf	fsr0
  1481  06E8  1383               	bcf	status, 7	;select IRP bank0
  1482  06E9  0800               	movf	indf,w
  1483  06EA  120A  118A  25AC   	fcall	_lcd_write
              120A  118A         
  1484                           opt subtitle "HI-TECH Software Omniscient Code Generator (Lite mode) build 49521"
  1485  06EF                     l999:	
  1486  06EF  120A  118A  2606   	fcall	_lcd_en
              120A  118A         
  1487                           opt subtitle "HI-TECH Software Omniscient Code Generator (Lite mode) build 49521"
  1488  06F4                     l1001:	
  1489  06F4  3001               	movlw	(01h)
  1490  06F5  00F5               	movwf	(??_lcd_printf+0)+0
  1491  06F6  0875               	movf	(??_lcd_printf+0)+0,w
  1492  06F7  07F6               	addwf	(lcd_printf@i),f
  1493                           opt subtitle "HI-TECH Software Omniscient Code Generator (Lite mode) build 49521"
  1494  06F8                     l1003:	
  1495  06F8  3010               	movlw	(010h)
  1496  06F9  0276               	subwf	(lcd_printf@i),w
  1497  06FA  1C03               	skipc
  1498  06FB  2EFD               	goto	u291
  1499  06FC  2EFE               	goto	u290
  1500  06FD                     u291:
  1501  06FD  2EE5               	goto	l997
  1502  06FE                     u290:
  1503  06FE  2EFF               	goto	l1005
  1504                           opt subtitle "HI-TECH Software Omniscient Code Generator (Lite mode) build 49521"
  1505  06FF                     l67:	
  1506                           opt subtitle "HI-TECH Software Omniscient Code Generator (Lite mode) build 49521"
  1507                           
  1508  06FF                     l1005:	
  1509                           opt subtitle "HI-TECH Software Omniscient Code Generator (Lite mode) build 49521"
  1510  06FF  3002               	movlw	(02h)
  1511  0700  120A  118A  269C   	fcall	_lcd_set_line
              120A  118A         
  1512                           opt subtitle "HI-TECH Software Omniscient Code Generator (Lite mode) build 49521"
  1513                           
  1514  0705                     l1007:	
  1515                           opt subtitle "HI-TECH Software Omniscient Code Generator (Lite mode) build 49521"
  1516  0705  01F6               	clrf	(lcd_printf@i)
  1517                           opt subtitle "HI-TECH Software Omniscient Code Generator (Lite mode) build 49521"
  1518  0706                     l1009:	
  1519  0706  3010               	movlw	(010h)
  1520  0707  0276               	subwf	(lcd_printf@i),w
  1521  0708  1C03               	skipc
  1522  0709  2F0B               	goto	u301
  1523  070A  2F0C               	goto	u300
  1524  070B                     u301:
  1525  070B  2F0E               	goto	l1013
  1526  070C                     u300:
  1527  070C  2F28               	goto	l70
  1528                           opt subtitle "HI-TECH Software Omniscient Code Generator (Lite mode) build 49521"
  1529  070D                     l1011:	
  1530  070D  2F28               	goto	l70
  1531                           opt subtitle "HI-TECH Software Omniscient Code Generator (Lite mode) build 49521"
  1532  070E                     l68:	
  1533                           opt subtitle "HI-TECH Software Omniscient Code Generator (Lite mode) build 49521"
  1534  070E                     l1013:	
  1535  070E  0876               	movf	(lcd_printf@i),w
  1536  070F  3E30               	addlw	_lcd_buffer_2&0ffh
  1537  0710  0084               	movwf	fsr0
  1538  0711  1383               	bcf	status, 7	;select IRP bank0
  1539  0712  0800               	movf	indf,w
  1540  0713  120A  118A  25AC   	fcall	_lcd_write
              120A  118A         
  1541                           opt subtitle "HI-TECH Software Omniscient Code Generator (Lite mode) build 49521"
  1542  0718                     l1015:	
  1543  0718  120A  118A  2606   	fcall	_lcd_en
              120A  118A         
  1544                           opt subtitle "HI-TECH Software Omniscient Code Generator (Lite mode) build 49521"
  1545  071D                     l1017:	
  1546  071D  3001               	movlw	(01h)
  1547  071E  00F5               	movwf	(??_lcd_printf+0)+0
  1548  071F  0875               	movf	(??_lcd_printf+0)+0,w
  1549  0720  07F6               	addwf	(lcd_printf@i),f
  1550                           opt subtitle "HI-TECH Software Omniscient Code Generator (Lite mode) build 49521"
  1551  0721                     l1019:	
  1552  0721  3010               	movlw	(010h)
  1553  0722  0276               	subwf	(lcd_printf@i),w
  1554  0723  1C03               	skipc
  1555  0724  2F26               	goto	u311
  1556  0725  2F27               	goto	u310
  1557  0726                     u311:
  1558  0726  2F0E               	goto	l1013
  1559  0727                     u310:
  1560  0727  2F28               	goto	l70
  1561                           opt subtitle "HI-TECH Software Omniscient Code Generator (Lite mode) build 49521"
  1562  0728                     l69:	
  1563                           opt subtitle "HI-TECH Software Omniscient Code Generator (Lite mode) build 49521"
  1564                           
  1565  0728                     l70:	
  1566  0728  0008               	return
  1567                           opt subtitle "HI-TECH Software Omniscient Code Generator (Lite mode) build 49521"
  1568                           
  1569  0729                     	__end_of_lcd_printf:
  1570                           opt subtitle "HI-TECH Software Omniscient Code Generator (Lite mode) build 49521"
  1571                           
  1572                           opt pagewidth 120
  1573                           
  1574                           	opt lm
  1575                           
  1576                           	processor	16F877A
  1577                           clrc	macro
  1578                           	bcf	3,0
  1579                           	endm
  1580                           clrz	macro
  1581                           	bcf	3,2
  1582                           	endm
  1583                           setc	macro
  1584                           	bsf	3,0
  1585                           	endm
  1586                           setz	macro
  1587                           	bsf	3,2
  1588                           	endm
  1589                           skipc	macro
  1590                           	btfss	3,0
  1591                           	endm
  1592                           skipz	macro
  1593                           	btfss	3,2
  1594                           	endm
  1595                           skipnc	macro
  1596                           	btfsc	3,0
  1597                           	endm
  1598                           skipnz	macro
  1599                           	btfsc	3,2
  1600                           	endm
  1601                           indf	equ	0
  1602                           indf0	equ	0
  1603                           pc	equ	2
  1604                           pcl	equ	2
  1605                           status	equ	3
  1606                           fsr	equ	4
  1607                           fsr0	equ	4
  1608                           c	equ	1
  1609  069C                     __ptext267:	;psect for function _lcd_set_line
  1610                           opt subtitle "HI-TECH Software Omniscient Code Generator (Lite mode) build 49521"
  1611                           
  1612                           opt pagewidth 120
  1613                           
  1614  0039                     	__size_of_lcd_set_line	equ	__end_of_lcd_set_line-_lcd_set_line
  1615                           opt subtitle "HI-TECH Software Omniscient Code Generator (Lite mode) build 49521"
  1616  069C                     _lcd_set_line:	
  1617                           opt subtitle "HI-TECH Software Omniscient Code Generator (Lite mode) build 49521"
  1618                           
  1619                           opt pagewidth 120
  1620  069C  00F4               	movwf	(lcd_set_line@line)
  1621                           opt subtitle "HI-TECH Software Omniscient Code Generator (Lite mode) build 49521"
  1622                           
  1623  069D                     l969:	
  1624                           opt subtitle "HI-TECH Software Omniscient Code Generator (Lite mode) build 49521"
  1625  069D  30E8               	movlw	low(03E8h)
  1626  069E  00F0               	movwf	(?_delay_us)
  1627  069F  3003               	movlw	high(03E8h)
  1628  06A0  00F1               	movwf	((?_delay_us))+1
  1629  06A1  120A  118A  2639   	fcall	_delay_us
              120A  118A         
  1630                           opt subtitle "HI-TECH Software Omniscient Code Generator (Lite mode) build 49521"
  1631                           
  1632  06A6                     l971:	
  1633                           opt subtitle "HI-TECH Software Omniscient Code Generator (Lite mode) build 49521"
  1634  06A6  120A  118A  25A8   	fcall	_lcd_cmd
              120A  118A         
  1635                           opt subtitle "HI-TECH Software Omniscient Code Generator (Lite mode) build 49521"
  1636                           
  1637  06AB                     l973:	
  1638                           opt subtitle "HI-TECH Software Omniscient Code Generator (Lite mode) build 49521"
  1639  06AB  3001               	movlw	(01h)
  1640  06AC  120A  118A  25DC   	fcall	_lcd_rw
              120A  118A         
  1641                           opt subtitle "HI-TECH Software Omniscient Code Generator (Lite mode) build 49521"
  1642                           
  1643  06B1  2EC2               	goto	l981
  1644                           opt subtitle "HI-TECH Software Omniscient Code Generator (Lite mode) build 49521"
  1645                           
  1646                           opt pagewidth 120
  1647                           
  1648  06B2                     l59:	
  1649                           opt subtitle "HI-TECH Software Omniscient Code Generator (Lite mode) build 49521"
  1650  06B2                     l975:	
  1651  06B2  3080               	movlw	(080h)
  1652  06B3  120A  118A  25AC   	fcall	_lcd_write
              120A  118A         
  1653  06B8  2ECA               	goto	l983
  1654                           opt subtitle "HI-TECH Software Omniscient Code Generator (Lite mode) build 49521"
  1655                           
  1656                           opt pagewidth 120
  1657  06B9                     l61:	
  1658                           opt subtitle "HI-TECH Software Omniscient Code Generator (Lite mode) build 49521"
  1659  06B9                     l977:	
  1660  06B9  30C0               	movlw	(0C0h)
  1661  06BA  120A  118A  25AC   	fcall	_lcd_write
              120A  118A         
  1662  06BF  2ECA               	goto	l983
  1663                           opt subtitle "HI-TECH Software Omniscient Code Generator (Lite mode) build 49521"
  1664                           
  1665                           opt pagewidth 120
  1666  06C0                     l62:	
  1667  06C0  2ECA               	goto	l983
  1668                           opt subtitle "HI-TECH Software Omniscient Code Generator (Lite mode) build 49521"
  1669                           
  1670  06C1                     l979:	
  1671                           opt subtitle "HI-TECH Software Omniscient Code Generator (Lite mode) build 49521"
  1672  06C1  2ECA               	goto	l983
  1673                           opt subtitle "HI-TECH Software Omniscient Code Generator (Lite mode) build 49521"
  1674                           
  1675  06C2                     l58:	
  1676                           opt subtitle "HI-TECH Software Omniscient Code Generator (Lite mode) build 49521"
  1677  06C2                     l981:	
  1678  06C2  0874               	movf	(lcd_set_line@line),w
  1679                           opt subtitle "HI-TECH Software Omniscient Code Generator (Lite mode) build 49521"
  1680                           
  1681                           opt pagewidth 120
  1682                           
  1683                           	opt lm
  1684                           
  1685                           	processor	16F877A
  1686                           clrc	macro
  1687                           	bcf	3,0
  1688                           	endm
  1689  06C3  3A01               	xorlw	1^0	; case 1
  1690  06C4  1903               	skipnz
  1691  06C5  2EB2               	goto	l975
  1692  06C6  3A03               	xorlw	2^1	; case 2
  1693  06C7  1903               	skipnz
  1694  06C8  2EB9               	goto	l977
  1695  06C9  2ECA               	goto	l983
  1696                           opt subtitle "HI-TECH Software Omniscient Code Generator (Lite mode) build 49521"
  1697                           
  1698                           opt pagewidth 120
  1699                           
  1700  06CA                     l60:	
  1701                           opt subtitle "HI-TECH Software Omniscient Code Generator (Lite mode) build 49521"
  1702                           
  1703  06CA                     l983:	
  1704                           opt subtitle "HI-TECH Software Omniscient Code Generator (Lite mode) build 49521"
  1705  06CA  120A  118A  2606   	fcall	_lcd_en
              120A  118A         
  1706                           opt subtitle "HI-TECH Software Omniscient Code Generator (Lite mode) build 49521"
  1707                           
  1708  06CF                     l985:	
  1709                           opt subtitle "HI-TECH Software Omniscient Code Generator (Lite mode) build 49521"
  1710  06CF  120A  118A  25A4   	fcall	_lcd_data
              120A  118A         
  1711                           opt subtitle "HI-TECH Software Omniscient Code Generator (Lite mode) build 49521"
  1712                           
  1713  06D4                     l63:	
  1714  06D4  0008               	return
  1715                           opt subtitle "HI-TECH Software Omniscient Code Generator (Lite mode) build 49521"
  1716                           
  1717  06D5                     	__end_of_lcd_set_line:
  1718                           opt subtitle "HI-TECH Software Omniscient Code Generator (Lite mode) build 49521"
  1719                           
  1720                           opt pagewidth 120
  1721                           
  1722                           	opt lm
  1723                           
  1724                           	processor	16F877A
  1725                           clrc	macro
  1726                           	bcf	3,0
  1727                           	endm
  1728                           clrz	macro
  1729                           	bcf	3,2
  1730                           	endm
  1731                           setc	macro
  1732                           	bsf	3,0
  1733                           	endm
  1734                           setz	macro
  1735                           	bsf	3,2
  1736                           	endm
  1737                           skipc	macro
  1738                           	btfss	3,0
  1739                           	endm
  1740                           skipz	macro
  1741                           	btfss	3,2
  1742                           	endm
  1743                           skipnc	macro
  1744                           	btfsc	3,0
  1745                           	endm
  1746                           skipnz	macro
  1747                           	btfsc	3,2
  1748                           	endm
  1749                           indf	equ	0
  1750                           indf0	equ	0
  1751                           pc	equ	2
  1752                           pcl	equ	2
  1753  05A8                     __ptext268:	;psect for function _lcd_cmd
  1754                           opt subtitle "HI-TECH Software Omniscient Code Generator (Lite mode) build 49521"
  1755                           
  1756                           opt pagewidth 120
  1757                           
  1758  0004                     	__size_of_lcd_cmd	equ	__end_of_lcd_cmd-_lcd_cmd
  1759                           opt subtitle "HI-TECH Software Omniscient Code Generator (Lite mode) build 49521"
  1760  05A8                     _lcd_cmd:	
  1761                           opt subtitle "HI-TECH Software Omniscient Code Generator (Lite mode) build 49521"
  1762                           
  1763                           opt pagewidth 120
  1764                           
  1765  05A8                     l823:	
  1766                           opt subtitle "HI-TECH Software Omniscient Code Generator (Lite mode) build 49521"
  1767  05A8  1283               	bcf	status, 5	;RP0=0, select bank0
  1768  05A9  1303               	bcf	status, 6	;RP1=0, select bank0
  1769  05AA  1006               	bcf	(6),0	;volatile
  1770                           opt subtitle "HI-TECH Software Omniscient Code Generator (Lite mode) build 49521"
  1771                           
  1772  05AB                     l41:	
  1773  05AB  0008               	return
  1774                           opt subtitle "HI-TECH Software Omniscient Code Generator (Lite mode) build 49521"
  1775                           
  1776  05AC                     	__end_of_lcd_cmd:
  1777                           opt subtitle "HI-TECH Software Omniscient Code Generator (Lite mode) build 49521"
  1778                           
  1779                           opt pagewidth 120
  1780                           
  1781                           	opt lm
  1782                           
  1783                           	processor	16F877A
  1784                           clrc	macro
  1785                           	bcf	3,0
  1786                           	endm
  1787                           clrz	macro
  1788                           	bcf	3,2
  1789                           	endm
  1790                           setc	macro
  1791                           	bsf	3,0
  1792                           	endm
  1793                           setz	macro
  1794                           	bsf	3,2
  1795                           	endm
  1796                           skipc	macro
  1797                           	btfss	3,0
  1798                           	endm
  1799                           skipz	macro
  1800                           	btfss	3,2
  1801                           	endm
  1802                           skipnc	macro
  1803                           	btfsc	3,0
  1804                           	endm
  1805                           skipnz	macro
  1806                           	btfsc	3,2
  1807                           	endm
  1808                           indf	equ	0
  1809                           indf0	equ	0
  1810                           pc	equ	2
  1811  05DC                     __ptext269:	;psect for function _lcd_rw
  1812                           opt subtitle "HI-TECH Software Omniscient Code Generator (Lite mode) build 49521"
  1813                           
  1814                           opt pagewidth 120
  1815                           
  1816  0015                     	__size_of_lcd_rw	equ	__end_of_lcd_rw-_lcd_rw
  1817                           opt subtitle "HI-TECH Software Omniscient Code Generator (Lite mode) build 49521"
  1818  05DC                     _lcd_rw:	
  1819                           opt subtitle "HI-TECH Software Omniscient Code Generator (Lite mode) build 49521"
  1820                           
  1821                           opt pagewidth 120
  1822  05DC  00F0               	movwf	(lcd_rw@sel)
  1823                           opt subtitle "HI-TECH Software Omniscient Code Generator (Lite mode) build 49521"
  1824                           
  1825  05DD                     l825:	
  1826                           opt subtitle "HI-TECH Software Omniscient Code Generator (Lite mode) build 49521"
  1827  05DD  2DE8               	goto	l829
  1828                           opt subtitle "HI-TECH Software Omniscient Code Generator (Lite mode) build 49521"
  1829                           
  1830                           opt pagewidth 120
  1831                           
  1832  05DE                     l48:	
  1833  05DE  1283               	bcf	status, 5	;RP0=0, select bank0
  1834  05DF  1303               	bcf	status, 6	;RP1=0, select bank0
  1835  05E0  1486               	bsf	(6),1	;volatile
  1836  05E1  2DF0               	goto	l52
  1837                           opt subtitle "HI-TECH Software Omniscient Code Generator (Lite mode) build 49521"
  1838                           
  1839                           opt pagewidth 120
  1840  05E2                     l50:	
  1841  05E2  1283               	bcf	status, 5	;RP0=0, select bank0
  1842  05E3  1303               	bcf	status, 6	;RP1=0, select bank0
  1843  05E4  1086               	bcf	(6),1	;volatile
  1844  05E5  2DF0               	goto	l52
  1845                           opt subtitle "HI-TECH Software Omniscient Code Generator (Lite mode) build 49521"
  1846                           
  1847                           opt pagewidth 120
  1848  05E6                     l51:	
  1849  05E6  2DF0               	goto	l52
  1850                           opt subtitle "HI-TECH Software Omniscient Code Generator (Lite mode) build 49521"
  1851                           
  1852  05E7                     l827:	
  1853                           opt subtitle "HI-TECH Software Omniscient Code Generator (Lite mode) build 49521"
  1854  05E7  2DF0               	goto	l52
  1855                           opt subtitle "HI-TECH Software Omniscient Code Generator (Lite mode) build 49521"
  1856                           
  1857  05E8                     l47:	
  1858                           opt subtitle "HI-TECH Software Omniscient Code Generator (Lite mode) build 49521"
  1859  05E8                     l829:	
  1860  05E8  0870               	movf	(lcd_rw@sel),w
  1861                           opt subtitle "HI-TECH Software Omniscient Code Generator (Lite mode) build 49521"
  1862                           
  1863                           opt pagewidth 120
  1864                           
  1865                           	opt lm
  1866                           
  1867                           	processor	16F877A
  1868                           clrc	macro
  1869                           	bcf	3,0
  1870                           	endm
  1871                           clrz	macro
  1872                           	bcf	3,2
  1873                           	endm
  1874  05E9  3A00               	xorlw	0^0	; case 0
  1875  05EA  1903               	skipnz
  1876  05EB  2DDE               	goto	l48
  1877  05EC  3A01               	xorlw	1^0	; case 1
  1878  05ED  1903               	skipnz
  1879  05EE  2DE2               	goto	l50
  1880  05EF  2DF0               	goto	l52
  1881                           opt subtitle "HI-TECH Software Omniscient Code Generator (Lite mode) build 49521"
  1882                           
  1883                           opt pagewidth 120
  1884                           
  1885  05F0                     l49:	
  1886                           opt subtitle "HI-TECH Software Omniscient Code Generator (Lite mode) build 49521"
  1887                           
  1888  05F0                     l52:	
  1889  05F0  0008               	return
  1890                           opt subtitle "HI-TECH Software Omniscient Code Generator (Lite mode) build 49521"
  1891                           
  1892  05F1                     	__end_of_lcd_rw:
  1893                           opt subtitle "HI-TECH Software Omniscient Code Generator (Lite mode) build 49521"
  1894                           
  1895                           opt pagewidth 120
  1896                           
  1897                           	opt lm
  1898                           
  1899                           	processor	16F877A
  1900                           clrc	macro
  1901                           	bcf	3,0
  1902                           	endm
  1903                           clrz	macro
  1904                           	bcf	3,2
  1905                           	endm
  1906                           setc	macro
  1907                           	bsf	3,0
  1908                           	endm
  1909                           setz	macro
  1910                           	bsf	3,2
  1911                           	endm
  1912                           skipc	macro
  1913                           	btfss	3,0
  1914                           	endm
  1915                           skipz	macro
  1916                           	btfss	3,2
  1917                           	endm
  1918                           skipnc	macro
  1919                           	btfsc	3,0
  1920                           	endm
  1921                           skipnz	macro
  1922                           	btfsc	3,2
  1923                           	endm
  1924                           indf	equ	0
  1925                           indf0	equ	0
  1926                           pc	equ	2
  1927                           pcl	equ	2
  1928                           status	equ	3
  1929  05AC                     __ptext270:	;psect for function _lcd_write
  1930                           opt subtitle "HI-TECH Software Omniscient Code Generator (Lite mode) build 49521"
  1931                           
  1932                           opt pagewidth 120
  1933                           
  1934  0006                     	__size_of_lcd_write	equ	__end_of_lcd_write-_lcd_write
  1935                           opt subtitle "HI-TECH Software Omniscient Code Generator (Lite mode) build 49521"
  1936  05AC                     _lcd_write:	
  1937                           opt subtitle "HI-TECH Software Omniscient Code Generator (Lite mode) build 49521"
  1938                           
  1939                           opt pagewidth 120
  1940                           
  1941  05AC  00F0               	movwf	(lcd_write@databuffer)
  1942                           opt subtitle "HI-TECH Software Omniscient Code Generator (Lite mode) build 49521"
  1943  05AD                     l831:	
  1944                           opt subtitle "HI-TECH Software Omniscient Code Generator (Lite mode) build 49521"
  1945  05AD  0870               	movf	(lcd_write@databuffer),w
  1946  05AE  1283               	bcf	status, 5	;RP0=0, select bank0
  1947  05AF  1303               	bcf	status, 6	;RP1=0, select bank0
  1948  05B0  0088               	movwf	(8)	;volatile
  1949                           opt subtitle "HI-TECH Software Omniscient Code Generator (Lite mode) build 49521"
  1950                           
  1951  05B1                     l55:	
  1952  05B1  0008               	return
  1953                           opt subtitle "HI-TECH Software Omniscient Code Generator (Lite mode) build 49521"
  1954                           
  1955  05B2                     	__end_of_lcd_write:
  1956                           opt subtitle "HI-TECH Software Omniscient Code Generator (Lite mode) build 49521"
  1957                           
  1958                           opt pagewidth 120
  1959                           
  1960                           	opt lm
  1961                           
  1962                           	processor	16F877A
  1963                           clrc	macro
  1964                           	bcf	3,0
  1965                           	endm
  1966                           clrz	macro
  1967                           	bcf	3,2
  1968                           	endm
  1969                           setc	macro
  1970                           	bsf	3,0
  1971                           	endm
  1972                           setz	macro
  1973                           	bsf	3,2
  1974                           	endm
  1975                           skipc	macro
  1976                           	btfss	3,0
  1977                           	endm
  1978                           skipz	macro
  1979                           	btfss	3,2
  1980                           	endm
  1981                           skipnc	macro
  1982                           	btfsc	3,0
  1983                           	endm
  1984                           skipnz	macro
  1985                           	btfsc	3,2
  1986                           	endm
  1987                           indf	equ	0
  1988                           indf0	equ	0
  1989                           pc	equ	2
  1990                           pcl	equ	2
  1991                           status	equ	3
  1992                           fsr	equ	4
  1993  0606                     __ptext271:	;psect for function _lcd_en
  1994                           opt subtitle "HI-TECH Software Omniscient Code Generator (Lite mode) build 49521"
  1995                           
  1996                           opt pagewidth 120
  1997                           
  1998  0019                     	__size_of_lcd_en	equ	__end_of_lcd_en-_lcd_en
  1999                           opt subtitle "HI-TECH Software Omniscient Code Generator (Lite mode) build 49521"
  2000  0606                     _lcd_en:	
  2001                           opt subtitle "HI-TECH Software Omniscient Code Generator (Lite mode) build 49521"
  2002                           
  2003                           opt pagewidth 120
  2004                           
  2005  0606                     l923:	
  2006                           opt subtitle "HI-TECH Software Omniscient Code Generator (Lite mode) build 49521"
  2007  0606  1283               	bcf	status, 5	;RP0=0, select bank0
  2008  0607  1303               	bcf	status, 6	;RP1=0, select bank0
  2009  0608  1506               	bsf	(6),2	;volatile
  2010                           opt subtitle "HI-TECH Software Omniscient Code Generator (Lite mode) build 49521"
  2011                           
  2012  0609                     l925:	
  2013                           opt subtitle "HI-TECH Software Omniscient Code Generator (Lite mode) build 49521"
  2014  0609  300A               	movlw	low(0Ah)
  2015  060A  00F0               	movwf	(?_delay_us)
  2016  060B  3000               	movlw	high(0Ah)
  2017  060C  00F1               	movwf	((?_delay_us))+1
  2018  060D  120A  118A  2639   	fcall	_delay_us
              120A  118A         
  2019                           opt subtitle "HI-TECH Software Omniscient Code Generator (Lite mode) build 49521"
  2020                           
  2021  0612                     l927:	
  2022                           opt subtitle "HI-TECH Software Omniscient Code Generator (Lite mode) build 49521"
  2023  0612  1283               	bcf	status, 5	;RP0=0, select bank0
  2024  0613  1303               	bcf	status, 6	;RP1=0, select bank0
  2025  0614  1106               	bcf	(6),2	;volatile
  2026                           opt subtitle "HI-TECH Software Omniscient Code Generator (Lite mode) build 49521"
  2027                           
  2028  0615  300A               	movlw	low(0Ah)
  2029  0616  00F0               	movwf	(?_delay_us)
  2030  0617  3000               	movlw	high(0Ah)
  2031  0618  00F1               	movwf	((?_delay_us))+1
  2032  0619  120A  118A  2639   	fcall	_delay_us
              120A  118A         
  2033                           opt subtitle "HI-TECH Software Omniscient Code Generator (Lite mode) build 49521"
  2034                           
  2035  061E                     l44:	
  2036  061E  0008               	return
  2037                           opt subtitle "HI-TECH Software Omniscient Code Generator (Lite mode) build 49521"
  2038                           
  2039  061F                     	__end_of_lcd_en:
  2040                           opt subtitle "HI-TECH Software Omniscient Code Generator (Lite mode) build 49521"
  2041                           
  2042                           opt pagewidth 120
  2043                           
  2044                           	opt lm
  2045                           
  2046                           	processor	16F877A
  2047                           clrc	macro
  2048                           	bcf	3,0
  2049                           	endm
  2050                           clrz	macro
  2051                           	bcf	3,2
  2052                           	endm
  2053                           setc	macro
  2054                           	bsf	3,0
  2055                           	endm
  2056                           setz	macro
  2057                           	bsf	3,2
  2058                           	endm
  2059                           skipc	macro
  2060                           	btfss	3,0
  2061                           	endm
  2062                           skipz	macro
  2063                           	btfss	3,2
  2064                           	endm
  2065                           skipnc	macro
  2066                           	btfsc	3,0
  2067                           	endm
  2068                           skipnz	macro
  2069                           	btfsc	3,2
  2070                           	endm
  2071                           indf	equ	0
  2072                           indf0	equ	0
  2073                           pc	equ	2
  2074                           pcl	equ	2
  2075  05A4                     __ptext272:	;psect for function _lcd_data
  2076                           opt subtitle "HI-TECH Software Omniscient Code Generator (Lite mode) build 49521"
  2077                           
  2078                           opt pagewidth 120
  2079                           
  2080  0004                     	__size_of_lcd_data	equ	__end_of_lcd_data-_lcd_data
  2081                           opt subtitle "HI-TECH Software Omniscient Code Generator (Lite mode) build 49521"
  2082  05A4                     _lcd_data:	
  2083                           opt subtitle "HI-TECH Software Omniscient Code Generator (Lite mode) build 49521"
  2084                           
  2085                           opt pagewidth 120
  2086                           
  2087  05A4                     l833:	
  2088                           opt subtitle "HI-TECH Software Omniscient Code Generator (Lite mode) build 49521"
  2089  05A4  1283               	bcf	status, 5	;RP0=0, select bank0
  2090  05A5  1303               	bcf	status, 6	;RP1=0, select bank0
  2091  05A6  1406               	bsf	(6),0	;volatile
  2092                           opt subtitle "HI-TECH Software Omniscient Code Generator (Lite mode) build 49521"
  2093                           
  2094  05A7                     l38:	
  2095  05A7  0008               	return
  2096                           opt subtitle "HI-TECH Software Omniscient Code Generator (Lite mode) build 49521"
  2097                           
  2098  05A8                     	__end_of_lcd_data:
  2099                           opt subtitle "HI-TECH Software Omniscient Code Generator (Lite mode) build 49521"
  2100                           
  2101                           opt pagewidth 120
  2102                           
  2103                           	opt lm
  2104                           
  2105                           	processor	16F877A
  2106                           clrc	macro
  2107                           	bcf	3,0
  2108                           	endm
  2109                           clrz	macro
  2110                           	bcf	3,2
  2111                           	endm
  2112                           setc	macro
  2113                           	bsf	3,0
  2114                           	endm
  2115                           setz	macro
  2116                           	bsf	3,2
  2117                           	endm
  2118                           skipc	macro
  2119                           	btfss	3,0
  2120                           	endm
  2121                           skipz	macro
  2122                           	btfss	3,2
  2123                           	endm
  2124                           skipnc	macro
  2125                           	btfsc	3,0
  2126                           	endm
  2127                           skipnz	macro
  2128                           	btfsc	3,2
  2129                           	endm
  2130                           indf	equ	0
  2131                           indf0	equ	0
  2132                           pc	equ	2
  2133  0639                     __ptext273:	;psect for function _delay_us
  2134                           opt subtitle "HI-TECH Software Omniscient Code Generator (Lite mode) build 49521"
  2135                           
  2136                           opt pagewidth 120
  2137                           
  2138  002B                     	__size_of_delay_us	equ	__end_of_delay_us-_delay_us
  2139                           opt subtitle "HI-TECH Software Omniscient Code Generator (Lite mode) build 49521"
  2140  0639                     _delay_us:	
  2141                           opt subtitle "HI-TECH Software Omniscient Code Generator (Lite mode) build 49521"
  2142                           
  2143                           opt pagewidth 120
  2144                           
  2145  0639                     l841:	
  2146                           opt subtitle "HI-TECH Software Omniscient Code Generator (Lite mode) build 49521"
  2147                           
  2148  0639  2E52               	goto	l847
  2149                           opt subtitle "HI-TECH Software Omniscient Code Generator (Lite mode) build 49521"
  2150  063A                     l125:	
  2151                           opt subtitle "HI-TECH Software Omniscient Code Generator (Lite mode) build 49521"
  2152                           
  2153  063A                     l843:	
  2154                           opt subtitle "HI-TECH Software Omniscient Code Generator (Lite mode) build 49521"
  2155                           
  2156  063A  3064               	movlw	low(064h)
  2157  063B  00F2               	movwf	(delay_us@i)
  2158  063C  3000               	movlw	high(064h)
  2159  063D  00F3               	movwf	((delay_us@i))+1
  2160                           opt subtitle "HI-TECH Software Omniscient Code Generator (Lite mode) build 49521"
  2161                           
  2162  063E  2E40               	goto	l845
  2163                           opt subtitle "HI-TECH Software Omniscient Code Generator (Lite mode) build 49521"
  2164  063F                     l127:	
  2165  063F  2E40               	goto	l845
  2166                           opt subtitle "HI-TECH Software Omniscient Code Generator (Lite mode) build 49521"
  2167  0640                     l126:	
  2168                           opt subtitle "HI-TECH Software Omniscient Code Generator (Lite mode) build 49521"
  2169  0640                     l845:	
  2170  0640  3001               	movlw	low(01h)
  2171  0641  02F2               	subwf	(delay_us@i),f
  2172  0642  3000               	movlw	high(01h)
  2173  0643  1C03               	skipc
  2174  0644  03F3               	decf	(delay_us@i+1),f
  2175  0645  02F3               	subwf	(delay_us@i+1),f
  2176  0646  30FF               	movlw	high(0FFFFh)
  2177  0647  0673               	xorwf	((delay_us@i+1)),w
  2178  0648  1D03               	skipz
  2179  0649  2E4C               	goto	u185
  2180  064A  30FF               	movlw	low(0FFFFh)
  2181  064B  0672               	xorwf	((delay_us@i)),w
  2182  064C                     u185:
  2183                           opt subtitle "HI-TECH Software Omniscient Code Generator (Lite mode) build 49521"
  2184  064C  1D03               	skipz
  2185  064D  2E4F               	goto	u181
  2186  064E  2E50               	goto	u180
  2187  064F                     u181:
  2188  064F  2E40               	goto	l845
  2189  0650                     u180:
  2190  0650  2E52               	goto	l847
  2191                           opt subtitle "HI-TECH Software Omniscient Code Generator (Lite mode) build 49521"
  2192  0651                     l128:	
  2193  0651  2E52               	goto	l847
  2194                           opt subtitle "HI-TECH Software Omniscient Code Generator (Lite mode) build 49521"
  2195                           
  2196  0652                     l124:	
  2197                           opt subtitle "HI-TECH Software Omniscient Code Generator (Lite mode) build 49521"
  2198                           
  2199  0652                     l847:	
  2200  0652  3001               	movlw	low(01h)
  2201  0653  02F0               	subwf	(delay_us@n),f
  2202  0654  3000               	movlw	high(01h)
  2203  0655  1C03               	skipc
  2204  0656  03F1               	decf	(delay_us@n+1),f
  2205  0657  02F1               	subwf	(delay_us@n+1),f
  2206  0658  30FF               	movlw	high(0FFFFh)
  2207  0659  0671               	xorwf	((delay_us@n+1)),w
  2208  065A  1D03               	skipz
  2209  065B  2E5E               	goto	u195
  2210  065C  30FF               	movlw	low(0FFFFh)
  2211  065D  0670               	xorwf	((delay_us@n)),w
  2212  065E                     u195:
  2213                           opt subtitle "HI-TECH Software Omniscient Code Generator (Lite mode) build 49521"
  2214  065E  1D03               	skipz
  2215  065F  2E61               	goto	u191
  2216  0660  2E62               	goto	u190
  2217  0661                     u191:
  2218  0661  2E3A               	goto	l843
  2219  0662                     u190:
  2220  0662  2E63               	goto	l130
  2221                           opt subtitle "HI-TECH Software Omniscient Code Generator (Lite mode) build 49521"
  2222  0663                     l129:	
  2223                           opt subtitle "HI-TECH Software Omniscient Code Generator (Lite mode) build 49521"
  2224                           
  2225  0663                     l130:	
  2226  0663  0008               	return
  2227                           opt subtitle "HI-TECH Software Omniscient Code Generator (Lite mode) build 49521"
  2228                           
  2229  0664                     	__end_of_delay_us:
  2230                           opt subtitle "HI-TECH Software Omniscient Code Generator (Lite mode) build 49521"
  2231                           
  2232                           opt pagewidth 120
  2233  0000                     __ptext274:	;psect for function _delay_us
  2234                           opt subtitle "HI-TECH Software Omniscient Code Generator (Lite mode) build 49521"
  2235  007E                     	btemp set 07Eh
  2236                           opt subtitle "HI-TECH Software Omniscient Code Generator (Lite mode) build 49521"
  2237                           
  2238                           opt pagewidth 120
  2239  007E                     	wtemp0 set btemp


Data Sizes:
    Strings     0
    Constant    0
    Data        15
    BSS         32
    Persistent  0
    Stack       0

Auto Spaces:
    Space          Size  Autos    Used
    COMMON           14     13      13
    BANK0            80     22      69
    BANK1            80      0       0
    BANK3            96      0       0
    BANK2            96      0       0

Pointer List with Targets:

    api_lcd_printf@databuffer	PTR unsigned char  size(1) Largest target is 15
		 -> main@test(BANK0[15]), 


Critical Paths under _main in COMMON

    _main->_api_lcd_printf
    _api_lcd_printf->_lcd_printf
    _lcd_printf->_lcd_set_line
    _lcd_set_line->_delay_us
    _lcd_en->_delay_us

Critical Paths under _main in BANK0

    _main->_api_lcd_printf

Critical Paths under _main in BANK1

    None.

Critical Paths under _main in BANK3

    None.

Critical Paths under _main in BANK2

    None.

Call Graph Tables:

 ---------------------------------------------------------------------------------
 (Depth) Function   	        Calls       Base Space   Used Autos Params    Refs
 ---------------------------------------------------------------------------------
 (0) _main                                                19    19      0     767
                                              3 BANK0     19    19      0
                 _api_lcd_initialize
                  _api_lcd_backlight
                     _api_lcd_printf
 ---------------------------------------------------------------------------------
 (1) _api_lcd_initialize                                   0     0      0      89
                            _lcd_cmd
                             _lcd_rw
                          _lcd_write
                             _lcd_en
                           _lcd_data
 ---------------------------------------------------------------------------------
 (1) _api_lcd_backlight                                    1     1      0      22
                                              0 COMMON     1     1      0
 ---------------------------------------------------------------------------------
 (1) _api_lcd_printf                                       9     6      3     631
                                              7 COMMON     6     3      3
                                              0 BANK0      3     3      0
                         _lcd_printf
 ---------------------------------------------------------------------------------
 (2) _lcd_printf                                           2     2      0     360
                                              5 COMMON     2     2      0
                       _lcd_set_line
                          _lcd_write
                             _lcd_en
 ---------------------------------------------------------------------------------
 (3) _lcd_set_line                                         1     1      0     156
                                              4 COMMON     1     1      0
                           _delay_us
                            _lcd_cmd
                             _lcd_rw
                          _lcd_write
                             _lcd_en
                           _lcd_data
 ---------------------------------------------------------------------------------
 (4) _lcd_cmd                                              0     0      0       0
 ---------------------------------------------------------------------------------
 (4) _lcd_rw                                               1     1      0      22
                                              0 COMMON     1     1      0
 ---------------------------------------------------------------------------------
 (3) _lcd_write                                            1     1      0      22
                                              0 COMMON     1     1      0
 ---------------------------------------------------------------------------------
 (3) _lcd_en                                               0     0      0      45
                           _delay_us
 ---------------------------------------------------------------------------------
 (4) _lcd_data                                             0     0      0       0
 ---------------------------------------------------------------------------------
 (4) _delay_us                                             4     2      2      45
                                              0 COMMON     4     2      2
 ---------------------------------------------------------------------------------
 Estimated maximum stack depth 4
 ---------------------------------------------------------------------------------

 Call Graph Graphs:

 _main (ROOT)
   _api_lcd_initialize
     _lcd_cmd
     _lcd_rw
     _lcd_write
     _lcd_en
       _delay_us
     _lcd_data
   _api_lcd_backlight
   _api_lcd_printf
     _lcd_printf
       _lcd_set_line
         _delay_us
         _lcd_cmd
         _lcd_rw
         _lcd_write
         _lcd_en
           _delay_us
         _lcd_data
       _lcd_write
       _lcd_en
         _delay_us

 Address spaces:
Name               Size   Autos  Total    Cost      Usage
BANK3               60      0       0       9        0.0%
BITBANK3            60      0       0       8        0.0%
SFR3                 0      0       0       4        0.0%
BITSFR3              0      0       0       4        0.0%
BANK2               60      0       0      11        0.0%
BITBANK2            60      0       0      10        0.0%
SFR2                 0      0       0       5        0.0%
BITSFR2              0      0       0       5        0.0%
BANK1               50      0       0       7        0.0%
BITBANK1            50      0       0       6        0.0%
SFR1                 0      0       0       2        0.0%
BITSFR1              0      0       0       2        0.0%
BANK0               50     16      45       5       86.3%
BITBANK0            50      0       0       4        0.0%
SFR0                 0      0       0       1        0.0%
BITSFR0              0      0       0       1        0.0%
COMMON               E      D       D       1       92.9%
BITCOMMON            E      0       0       0        0.0%
CODE                 0      0       0       0        0.0%
DATA                 0      0      57      12        0.0%
ABS                  0      0      52       3        0.0%
NULL                 0      0       0       0        0.0%
STACK                0      0       5       2        0.0%
EEDATA             100      0       0       0        0.0%


Microchip Technology PIC Macro Assembler V1.12 build 49521 
Symbol Table                                                                                   Tue Dec 30 21:05:02 2014

                          pc 0002                ?_lcd_set_line 0070                  __CFG_CP$OFF 0000  
                         l30 05FD                           l31 05F3                           l32 0605  
                         l41 05AB                           l33 05F7                           l50 05E2  
                         l34 05FB                           l51 05E6                           l35 0605  
                         l27 0782                           l44 061E                           l52 05F0  
                         l60 06CA                           l61 06B9                           l38 05A7  
                         l62 06C0                           l70 0728                           l55 05B1  
                         l47 05E8                           l63 06D4                           l48 05DE  
                         l80 07A7                           l49 05F0                           l81 078F  
                         l58 06C2                           l66 06E5                           l82 07BC  
                         l59 06B2                           l67 06FF                           l83 07FA  
                         l68 070E                           l84 07BD                           l69 0728  
                         l85 07D6                           l78 07F0                           l86 07BE  
                         l87 07ED                           l79 078E                           l88 07EE  
                         l89 07FF                           fsr 0004                  __CFG_LVP$ON 0000  
                        l120 0699                          l121 0699                          l130 0663  
                        l124 0652                          l125 063A                          l126 0640  
                        l118 0698                          l127 063F                          l119 0698  
                        l128 0651                          l129 0663                          l831 05AD  
                        l823 05A8                          l841 0639                          l833 05A4  
                        l825 05DD                          l843 063A                          l923 0606  
                        l827 05E7                          l835 05F2                          l931 072F  
                        l845 0640                          l925 0609                          l829 05E8  
                        l837 05FC                          l941 0737                          l933 0730  
                        l847 0652                          l927 0612                          l839 05FD  
                        l951 0752                          l943 073C                          l935 0733  
                        l961 076D                          l953 0757                          l945 0742  
                        l937 0734                          l929 0729                          l971 06A6  
                        l963 0772                          l955 075C                          l947 0748  
                        l939 0735                          l981 06C2                          l973 06AB  
                        l965 0778                          l957 0762                          l949 074D  
                        l983 06CA                          l975 06B2                          l991 06DC  
                        l967 077D                          l959 0767                          l985 06CF  
                        l977 06B9                          l969 069D                          l993 06DD  
                        l979 06C1                          l995 06E4                          l987 06D5  
                        l997 06E5                          l989 06D6                          l999 06EF  
                        u300 070C                          u301 070B                          u310 0727  
                        u311 0726                          u320 07BB                          u321 07BA  
                        u330 07EC                          u331 07EB                          u180 0650  
                        u340 066E                          u181 064F                          u325 07B7  
                        u190 0662                          u191 0661                          u335 07E8  
                        u280 06E3                          u185 064C                          u281 06E2  
                        u290 06FE                 __CFG_CPD$OFF 0000                          u195 065E  
                        u291 06FD                          fsr0 0004                          indf 0000  
               __CFG_FOSC$XT 0000                         l1001 06F4                         l1011 070D  
                       l1003 06F8                         l1013 070E                         l1005 06FF  
                       l1021 0786                         l1015 0718                         l1007 0705  
                       l1031 07A7                         l1023 0788                         l1017 071D  
                       l1009 0706                         l1041 07EF                         l1033 07BE  
                       l1025 078F                         l1019 0721                         l1035 07CD  
                       l1027 079E                         l1043 07F0                         l1051 0680  
                       l1037 07D1                         l1045 07FA                         l1029 07A2  
                       l1053 0686                         l1039 07D6                         l1047 0664  
                       l1049 067B                 __CFG_WRT$OFF 0000                  lcd_printf@i 0076  
                       _main 0664                         btemp 007E                         start 0000  
             ??_lcd_set_line 0074                        ?_main 0070                __CFG_WDTE$OFF 0000  
 __size_of_api_lcd_backlight 0015                        _PORTD 0008                        _TRISD 0088  
            __end_of_lcd_cmd 05AC               __CFG_BOREN$OFF 0000                        pclath 000A  
                      status 0003                        wtemp0 007E              __initialization 061F  
               __end_of_main 069C                       ??_main 0043      __size_of_api_lcd_printf 007D  
           __end_of_delay_us 0664               __CFG_PWRTE$OFF 0000             __end_of_lcd_data 05A8  
                     _lcd_en 0606                       _lcd_rw 05DC                    ??_lcd_cmd 0070  
                     clrloop 05B3         __end_of_lcd_set_line 06D5      __end_of__initialization 0635  
        lcd_write@databuffer 0070               __pcstackCOMMON 0070                 __pidataBANK0 05BA  
         __size_of_lcd_write 0006  __size_of_api_lcd_initialize 005A                   __pbssBANK0 0020  
                 __pmaintext 0664                      ?_lcd_en 0070                      ?_lcd_rw 0070  
                  ?_delay_us 0070                   _lcd_printf 06D5                    ?_lcd_data 0070  
             _api_lcd_printf 0783            __end_of_lcd_write 05B2              __size_of_lcd_en 0019  
            __size_of_lcd_rw 0015                      _lcd_cmd 05A8        __size_of_lcd_set_line 0039  
                 ??_delay_us 0072       __end_of_api_lcd_printf 0800                   ??_lcd_data 0070  
       end_of_initialization 0635             lcd_set_line@line 0074                      init_ram 05CD  
               _lcd_buffer_1 0020                 _lcd_buffer_2 0030                 _lcd_set_line 069C  
                  _PORTBbits 0006                    _TRISBbits 0086              ?_api_lcd_printf 0077  
                ?_lcd_printf 0070         api_lcd_printf@cursor 0077               __end_of_lcd_en 061F  
             __end_of_lcd_rw 05F1          start_initialization 061F              api_lcd_printf@i 0041  
            api_lcd_printf@j 0042          __size_of_lcd_printf 0054                     ??_lcd_en 0074  
                   ??_lcd_rw 0070                  __pdataBANK0 0056       api_lcd_backlight@state 0070  
              __pcstackBANK0 0040   __end_of_api_lcd_initialize 0783           api_lcd_printf@line 0040  
          __size_of_delay_us 002B            __size_of_lcd_data 0004                    __ptext270 05AC  
                  __ptext271 0606                    __ptext263 0729                    __ptext272 05A4  
                  __ptext264 05F1                    __ptext273 0639                    __ptext265 0783  
                  __ptext274 0000                    __ptext266 06D5                    __ptext267 069C  
                  __ptext268 05A8                    __ptext269 05DC     api_lcd_printf@databuffer 0078  
                   ?_lcd_cmd 0070                    _lcd_write 05AC                    delay_us@i 0072  
                  delay_us@n 0070                    main@F1287 0056             ??_api_lcd_printf 007A  
                 ?_lcd_write 0070                    lcd_rw@sel 0070                 ??_lcd_printf 0075  
                  init_fetch 05C9           __end_of_lcd_printf 0729             __size_of_lcd_cmd 0004  
                   _delay_us 0639                     _lcd_data 05A4                __size_of_main 0038  
                   clear_ram 05B2                     main@test 0047                  ??_lcd_write 0070  
          _api_lcd_backlight 05F1           ?_api_lcd_backlight 0070          ??_api_lcd_backlight 0070  
         _api_lcd_initialize 0729    api_lcd_printf@data_length 0079          ?_api_lcd_initialize 0070  
  __end_of_api_lcd_backlight 0606         ??_api_lcd_initialize 0074  
